:020000040000FA
:080000000002040000000000F2
:020000040000FA
:040008004C030000A5
:020000040000FA
:04000C004C030000A1
:020000040000FA
:040010004C0300009D
:020000040000FA
:040014004C03000099
:020000040000FA
:040018004C03000095
:020000040000FA
:04001C004C03000091
:020000040000FA
:040020004C0300008D
:020000040000FA
:040024004C03000089
:020000040000FA
:040028004C03000085
:020000040000FA
:04002C004C03000081
:020000040000FA
:040030004C0300007D
:020000040000FA
:040034004C03000079
:020000040000FA
:040038004C03000075
:020000040000FA
:04003C004C03000071
:020000040000FA
:040040004C0300006D
:020000040000FA
:040044004C03000069
:020000040000FA
:040048004C03000065
:020000040000FA
:04004C004C03000061
:020000040000FA
:040050004C0300005D
:020000040000FA
:040054003A55000019
:020000040000FA
:040058005C550000F3
:020000040000FA
:04005C004C03000051
:020000040000FA
:040060004C0300004D
:020000040000FA
:040064004C03000049
:020000040000FA
:040068004C03000045
:020000040000FA
:04006C004C03000041
:020000040000FA
:040070004C0300003D
:020000040000FA
:040074004C03000039
:020000040000FA
:040078004C03000035
:020000040000FA
:04007C004C03000031
:020000040000FA
:040080004C0300002D
:020000040000FA
:040084004C03000029
:020000040000FA
:040088004C03000025
:020000040000FA
:04008C004C03000021
:020000040000FA
:040090004C0300001D
:020000040000FA
:040094004C03000019
:020000040000FA
:040098004C03000015
:020000040000FA
:04009C004C03000011
:020000040000FA
:0400A0004C0300000D
:020000040000FA
:0400A4004C03000009
:020000040000FA
:0400A8004C03000005
:020000040000FA
:0400AC004C03000001
:020000040000FA
:0400B0004C030000FD
:020000040000FA
:0400B4004C030000F9
:020000040000FA
:0400B8004C030000F5
:020000040000FA
:0400BC004C030000F1
:020000040000FA
:0400C0004C030000ED
:020000040000FA
:0400C4004C030000E9
:020000040000FA
:0400C8004C030000E5
:020000040000FA
:0400CC004C030000E1
:020000040000FA
:0400D0004C030000DD
:020000040000FA
:0400D4004C030000D9
:020000040000FA
:0400D8004C030000D5
:020000040000FA
:0400DC004C030000D1
:020000040000FA
:0400E0004C030000CD
:020000040000FA
:0400E4004C030000C9
:020000040000FA
:0400E8004C030000C5
:020000040000FA
:0400EC004C030000C1
:020000040000FA
:0400F0004C030000BD
:020000040000FA
:0400F4004C030000B9
:020000040000FA
:0400F8004C030000B5
:020000040000FA
:0400FC004C030000B1
:020000040000FA
:040100004C030000AC
:020000040000FA
:040104004C030000A8
:020000040000FA
:040108004C030000A4
:020000040000FA
:04010C004C030000A0
:020000040000FA
:040110004C0300009C
:020000040000FA
:040114004C03000098
:020000040000FA
:040118004C03000094
:020000040000FA
:04011C004C03000090
:020000040000FA
:040120004C0300008C
:020000040000FA
:040124004C03000088
:020000040000FA
:040128004C03000084
:020000040000FA
:04012C004C03000080
:020000040000FA
:040130004C0300007C
:020000040000FA
:040134004C03000078
:020000040000FA
:040138004C03000074
:020000040000FA
:04013C004C03000070
:020000040000FA
:040140004C0300006C
:020000040000FA
:040144004C03000068
:020000040000FA
:040148004C03000064
:020000040000FA
:040208004C030000A3
:020000040000FA
:04020C004C0300009F
:020000040000FA
:040210004C0300009B
:020000040000FA
:040214004C03000097
:020000040000FA
:040218004C03000093
:020000040000FA
:04021C004C0300008F
:020000040000FA
:040220004C0300008B
:020000040000FA
:040224004C03000087
:020000040000FA
:040228004C03000083
:020000040000FA
:04022C004C0300007F
:020000040000FA
:040230004C0300007B
:020000040000FA
:040234004C03000077
:020000040000FA
:040238004C03000073
:020000040000FA
:04023C004C0300006F
:020000040000FA
:040240004C0300006B
:020000040000FA
:040244004C03000067
:020000040000FA
:040248004C03000063
:020000040000FA
:04024C004C0300005F
:020000040000FA
:040250004C0300005B
:020000040000FA
:040254004C03000057
:020000040000FA
:040258004C03000053
:020000040000FA
:04025C004C0300004F
:020000040000FA
:040260004C0300004B
:020000040000FA
:040264004C03000047
:020000040000FA
:040268004C03000043
:020000040000FA
:04026C004C0300003F
:020000040000FA
:040270004C0300003B
:020000040000FA
:040274004C03000037
:020000040000FA
:040278004C03000033
:020000040000FA
:04027C004C0300002F
:020000040000FA
:040280004C0300002B
:020000040000FA
:040284004C03000027
:020000040000FA
:040288004C03000023
:020000040000FA
:04028C004C0300001F
:020000040000FA
:040290004C0300001B
:020000040000FA
:040294004C03000017
:020000040000FA
:040298004C03000013
:020000040000FA
:04029C004C0300000F
:020000040000FA
:0402A0004C0300000B
:020000040000FA
:0402A4004C03000007
:020000040000FA
:0402A8004C03000003
:020000040000FA
:0402AC004C030000FF
:020000040000FA
:0402B0004C030000FB
:020000040000FA
:0402B4004C030000F7
:020000040000FA
:0402B8004C030000F3
:020000040000FA
:0402BC004C030000EF
:020000040000FA
:0402C0004C030000EB
:020000040000FA
:0402C4004C030000E7
:020000040000FA
:0402C8004C030000E3
:020000040000FA
:0402CC004C030000DF
:020000040000FA
:0402D0004C030000DB
:020000040000FA
:0402D4004C030000D7
:020000040000FA
:0402D8004C030000D3
:020000040000FA
:0402DC004C030000CF
:020000040000FA
:0402E0004C030000CB
:020000040000FA
:0402E4004C030000C7
:020000040000FA
:0402E8004C030000C3
:020000040000FA
:0402EC004C030000BF
:020000040000FA
:0402F0004C030000BB
:020000040000FA
:0402F4004C030000B7
:020000040000FA
:0402F8004C030000B3
:020000040000FA
:0402FC004C030000AF
:020000040000FA
:040300004C030000AA
:020000040000FA
:040304004C030000A6
:020000040000FA
:040308004C030000A2
:020000040000FA
:04030C004C0300009E
:020000040000FA
:040310004C0300009A
:020000040000FA
:040314004C03000096
:020000040000FA
:040318004C03000092
:020000040000FA
:04031C004C0300008E
:020000040000FA
:040320004C0300008A
:020000040000FA
:040324004C03000086
:020000040000FA
:040328004C03000082
:020000040000FA
:04032C004C0300007E
:020000040000FA
:040330004C0300007A
:020000040000FA
:040334004C03000076
:020000040000FA
:040338004C03000072
:020000040000FA
:04033C004C0300006E
:020000040000FA
:040340004C0300006A
:020000040000FA
:040344004C03000066
:020000040000FA
:040348004C03000062
:020000040000FA
:10040000CFA221000E7F22000E0188000000000014
:10041000000020000000E000020032000001200087
:10042000200288000C0007008049260001002000FF
:1004300011000700000020000000E0000200320070
:100440000000020000000000206702000000000021
:100450000040DA000000FE004440A900002B20000C
:100460000000E0000300320000002000A00188002E
:100470004440A80000000600910188008000780038
:100480000000EB0015003700E280400032A0B4000D
:100490009101BA00E280400032A0B4009102BA009B
:1004A000E280400032A0B4000002EB00472BDE00E7
:1004B000F507B200602CE10004003A000059EB009F
:1004C0008301E900FDFF3E00040037006128E100E0
:1004D000010032000082EB000B00070011C3BA00DC
:1004E0001101BA000604E00003003A000200E00037
:1004F000E5FF3A0000000600F607B200960188000A
:1005000082007800F5FF37003159BA008301E90015
:100510000C0032002159BA008301E90008003200C2
:100520000400E00003003A00E280400032A0B40082
:10053000F5FF370011D9BA008301E900FAFF3A004C
:100540008100E800E180400032A0B4000000060015
:10055000000000000000000000000000000000009B
:10056000000000000000000000000000000000008B
:10057000000000000000000000000000000000007B
:10058000000000000000000000000000000000006B
:10059000000000000000000000000000000000005B
:1005A000000000000000000000000000000000004B
:1005B000000000000000000000000000000000003B
:1005C000000000000000000000000000000000002B
:1005D000000000000000000000000000000000001B
:1005E000000000000000000000000000000000000B
:1005F00000000000000000000000000000000000FB
:1006000000000000000000000000000000000000EA
:1006100000000000000000000000000000000000DA
:1006200000000000000000000000000000000000CA
:1006300000000000000000000000000000000000BA
:1006400000000000000000000000000000000000AA
:10065000000000000000000000000000000000009A
:10066000000000000000000000000000000000008A
:10067000000000000000000000000000000000007A
:10068000000000000000000000000000000000006A
:1006900000000000000000000040DA000000FE0042
:1006A00003F0A200889FBE008A9FBE008C1F7800C6
:1006B0004A010700510133006450E1004F0032004D
:1006C0006420E1005200320003826C0007003B000E
:1006D0000905D0000306D000820F54000C065D000F
:1006E0000200390002003200890178000306780018
:1006F0008582550004003D000003FD008103FD00DC
:100700008502EA008B854200840F720002003B00E4
:1007100060001000E08018006011B8000005EB00D8
:100720007A28E1000A00390006007800C75DDD0084
:10073000F707B200878075002D00370082817100B5
:100740000A017800610560008180D1000080D3003B
:100750008502E900F9FF3B00060440008784480059
:1007600002003B0060041400E0841C000988A30020
:10077000070032008A81710082817100610164008A
:100780008904D1000884D3008B05E80017003700E6
:100790000978A30013003A000B00E00013003400B6
:1007A0008B05E9000804440089844C000A44740065
:1007B0000978A3000D003A000B00E00007003400A8
:1007C0008B05E9000804440089844C0001003A00CC
:1007D0000B0020000978A300F7FF32000001EB00B6
:1007E00002003700828171000A017800C000070012
:1007F0000CF0A70001F0A000090137006420E1001F
:1008000002003A00838F6C00090133000801BE002A
:100810000200BE0002013700889FBE008A9FBE0012
:100820008C1F7800ED000700F400330003866C0095
:100830006450E1002E0032006420E10033003200F9
:100840006150E1002F0032006120E10031003200F0
:1008500085855500EB07B000090020000804200042
:10086000050037000804440089844C000A00310068
:100870000603430087834B000001530081815B0026
:10088000F8FF33000203BE000800A0000804440083
:1008900089844C00F6FF3900C639DD0083017300FE
:1008A00001003200130020008904D1000884D30025
:1008B0000998A300050032000800A7000300A0006B
:1008C0008904D1000884D3008B05E8008904D10095
:1008D0000884D3000001EB000281D20084000700ED
:1008E00001F0A1000CF0A70001F0A000CC0037003F
:1008F0006420E100CE0032000801BE000200BE000C
:10090000F7FF37006120E100C90032006000B80045
:10091000F3FF37000000200001F82700F0FF370048
:100920001400200014023700F4FF2F0012023700D9
:100930000003BE00940007006011B8000470A70017
:1009400007F0A10007F8A30017003A006509B100FD
:100950000D0032000D003500860220000628E1005F
:1009600003003500030028006000B8000200050005
:100970000000400081804800020149008381490055
:100980008502E900FAFF3A0000000600F88F4200F5
:10099000050034008100D1000080D3008502E8000A
:1009A000FCFF3A00000006006011B8008000EB0078
:1009B000000005000001BE00730007000470A700DE
:1009C00003F0A10003F8A30013003A006509B10089
:1009D00010003200090035006928E10002003500EE
:1009E0000100280000000500000040008180480050
:1009F0008502E900FCFF3A0000000600F88F420083
:100A0000050035008100D1000080D3008502E80098
:100A1000FCFF3A00000006008000EB00000005002B
:100A20004F89DE0082017800EE013700889FBE000A
:100A30008A9FBE000082700004027100048271006F
:100A4000260032000004BE000200BE006011B800A3
:100A50006B092000950220000182CF000A003900B6
:100A60000541B1000082CF00070039000541B10007
:100A70000982CF00040039000541B1000882CF008F
:100A8000010039000541B100054252001200320058
:100A90000A003B0082817100610164008100D10085
:100AA0000080D3008984D3000884D3008B05E8003C
:100AB0000442E800F7FF3A0007003700080444004A
:100AC00089844C0000004800818048008B05E900C3
:100AD0000442E900F9FF3A00050007004F05BE0097
:100AE0004F04BE00000006006011B800CFFF3700C1
:100AF00081002000618055000B003D000B002000AC
:100B000061FE2F000100E1001D00340082817100B0
:100B1000610164008904D1000884D3000000E8006A
:100B2000FAFF3A00710020006100640003007000C9
:100B3000020060000900320061044400E0844C00BF
:100B40000988A500050032008B05E8006808E1006F
:100B500002003A008904D1000884D300F20F20007B
:100B60000258E10005003D00C75DDD00F907B20055
:100B70008980750008007800000006000BF8270047
:100B80008B00780000000500C70ADE00F107B20004
:100B9000F50FB20008003200E1CF4200020032003F
:100BA0000170A00024000500810F700001003200D8
:100BB0000408050044000500810F700002003A009F
:100BC000140005008502E9000000400081C04800D3
:100BD000FCFF3B000170A000240005000004BE00E3
:100BE000E9FF07000003BE000405BE000200BE00CE
:100BF000E5FF0700844F7500000006000200BE00FC
:100C00006450E100050036006420E1000200360077
:100C10000968A30001003A000800BE000160A000BE
:100C20004F0678004F05BE004F04BE0000000600CE
:100C3000F0FF2F00F1FF2700F9FF3700889FBE006B
:100C40008A9FBE008C1F7800E4FF0700EBFF330093
:100C500003866C006450E100240032006420E1004F
:100C6000270032006150E100220032006120E100E3
:100C7000210032008B854200EB07B1000134B8003F
:100C8000003AB8000804420089844A00013AB800DA
:100C90000030B8008880400009014A000400330099
:100CA0000000400081804800020149008B05E900F6
:100CB000C909DD008301700001003200130020002B
:100CC000C814DE004814DD004709DE001200B2003F
:100CD000C808DE000884700085FF070001F0A1004D
:100CE0000CF0A70001F0A000CDFF37006120E1006B
:100CF000CFFF32000801BE000200BE00F7FF370040
:100D00006150E100FCFF3A00C9FF37006022B800E3
:100D1000060220000000D0008180D2000482D200B0
:100D20008582D2000000A0000202520083825A0095
:100D3000030031000202420083824A000000A10049
:100D40000603E900F3FF3A0000000600EFFF07008A
:100D50000400BE0000000600020AB900001BB90032
:100D60000200B8008100420081004300000006003C
:100D7000889FBE008A9FBE0030044200B0844A00B3
:100D800030054B0090854B006000B1000898BE0014
:100D90000A90BE000440E10005C8E10006D0E10071
:100DA00007D8E10002003100680040001008E800A8
:100DB0004F05BE004F04BE0000000600889FBE0025
:100DC0008A9FBE003004BE002005BE0004185400F7
:100DD00005985C0006185D0007985D001100200072
:100DE0000440E10005C8E10006D0E10007D8E100B9
:100DF000010039008000EB00108810004F05BE0094
:100E00004F04BE00000006001200FA00889FBE00DA
:100E10008A9FBE008C9FBE00E0B79F00F1B79F0085
:100E200082BF9F0093BF9F000605BE000404BE0062
:100E30000000EB00D0B79F00C0B79F00B0B79F0085
:100E4000A0B79F0090B79F000006EB005FB197002E
:100E5000CFB09700820141003FB097000200E00050
:100E600004003D00370007007E805700C0FF0700E8
:100E700003003700330007007E805700CFFF0700D4
:100E8000DFB697000D00E0000C0035006FB2970050
:100E9000FFB297000FBB97009FBB97001000200088
:100EA000010020006011B80000027200818272000F
:100EB00002037300838373001B0007000C06E80025
:100EC00001042000810F5600E0FF3A000D00E00011
:100ED00004003D000802BE000A03BE007E805700E9
:100EE000A3FF07005FA897000000E00005003A009C
:100EF0001FB29700AFB297003FB39700CFB39700F0
:100F0000090007006FB09700FFB097000FB9970076
:100F10009FB997004F06BE004F05BE004F04BE00AC
:100F20000080FA0000000600010007000000060033
:100F3000A4B79F00B5B79F00C6B79F00D7B79F0063
:100F4000000006004F09DE0082817100B3B79F00E8
:100F50004F01DE008180400082807000A1B79F00B9
:100F60008FB097004F09DE000000400002007000C3
:100F700090B79F007FA897004F01DE00818040005E
:100F80008280700081B79F000D0007004F3ADE009D
:100F90000000400004007000F0AF9F000800070050
:100FA0000402420085824A0006034B0087834B00FF
:100FB000DFFF07000802BE000A03BE0000000600B3
:100FC0002FB29700BFB297004FB39700DFB39700DF
:100FD00000000600881F780018002000881F780095
:100FE00089FF07008F87E9004F04780000000600A2
:100FF000801FEB0084FF07008F87E90000000600D8
:10100000889FBE008A9FBE00E00F5000E08F58000E
:10101000E00F5900E08F59000C003D006044B8001B
:101020006055B8000000540081805C0002015D0042
:1010300083815D00180020001500070008003D00B6
:10104000180007000004EB00050037000004EB0067
:101050000F00070002003D001200070018002000EA
:10106000DCFF07000800E000060032006022B80044
:101070006033B8000000520081805A0002015B001A
:1010800083815B004F05BE004F04BE0000000600D8
:10109000E00F5200E08F5A00E00F5B00E08F5B0032
:1010A000000006006044B8006055B8000402540017
:1010B00085825C0006035D0087835D0000000600FA
:1010C000889FBE008A9FBE008C1F7800E00F5000F2
:1010D000E08F5800E00F5900E08F59000D003D00EF
:1010E0006044B8006055B8000000540081805C0086
:1010F00002015D0083815D001C0020000820E100EA
:1011000009A8E1000AB0E1000BB8E1000D003D00C4
:10111000080037000006EB00E00F5200E08F5A0095
:10112000E00F5B00E08F5B0006003D006044B8000C
:101130006055B8000402540085825C0006035D001F
:1011400087835D00AAFF07000C00E0000600320064
:101150006022B8006033B8000000520081805A005D
:1011600002015B0083815B004F0678004F05BE00E3
:101170004F04BE0000000600889FBE008A9FBE008C
:10118000841F780095FE07004F007800110033009F
:10119000F0FF2F00838F6C0006003B000405650004
:1011A0000A00A7000800370009F0A6001000200080
:1011B00008003700820F5400838F5C000300390061
:1011C0001000200001003E000000200009F0A700F0
:1011D0000000EA004F05BE004F04BE000000E00022
:1011E00000000600881F7800030478000300E00078
:1011F00007003D0060001000E08018006001190049
:10120000E081190002003B0001F02D0003003700CF
:1012100006FE070008F0A70001F0A0004F047800C8
:0412200000000600C4
:020000040000FA
:101224000D0A00002800000078000000293E00009C
:101234000008000020080000000000002E2000002C
:1012440000200000004300006C750000746300007F
:101254006820000064690000736500006E67000088
:101264006167000065640000212100002100000086
:10127400546F000020660000696E0000697300006E
:10128400682000007365000074750000702C000075
:101294002073000074610000727400002075000067
:1012A400702000007468000065200000706F00006A
:1012B40077650000722000007375000070700000F4
:1012C4006C690000657300002077000069740000F9
:1012D40068200000636F00006D6D0000616E000007
:1012E4006420000027570000270D00000A000000BA
:1012F4004275000073200000506900007261000014
:1013040074650000207600003300000020630000B4
:101314006C6F00006E650000207700002F640000F1
:101324006966000066650000726500006E74000066
:101334002050000049430000004300006F6D00008E
:101344006D7500006E69000074790000204600008D
:10135400697200006D770000617200006520000072
:10136400763700002E300000202D0000206700009A
:101374006F6F00002E6700006C2F000067430000B1
:101384007A5100006E570000200000002028000061
:1013940032340000464A0000363400004741000061
:1013A4003030000000340000200000003220000033
:1013B40000410000330000004234000000420000FD
:1013C4003500000042380000005500004E4B00007C
:1013D4000029000000490000090000004F09000036
:1013E40000480000090000004C090000004500000E
:1013F4006E740000657200002072000061770000C6
:1014040020760000616C0000756500002066000015
:101414006F7200002042000052470000003E0000AE
:10142400001B00005B440000001B00005B00000088
:10143400440000001B5B0000430000001B5B000035
:10144400324B00000D000000430000001B5B000055
:101454003244000000570000617200006E69000011
:101464006E6700003A2000006E6F000020760000D6
:101474006F6C00007461000067650000206F00005D
:101484006E20000056700000756C00006C75000042
:1014940070200000706900006E000000203D000014
:1014A40020000000436C00007574000063680000B5
:1014B400206500006E67000061670000656400003D
:1014C4002121000021000000565200004547000081
:1014D400207400006F6F0000206C00006F77000024
:1014E4002C2000006973000020740000686500006F
:1014F400726500002061000020730000686F000026
:10150400727400003F0000002E2000003C00000028
:101514000041000052540000310000001434000067
:10152400040D00008206000040030000A00100003A
:10153400CF0000007F0000006700000044000000AE
:101544002200000000000000000000002C01000048
:10155400000000005802000000000000B004000079
:10156400000000006009000000000000C01200003C
:10157400000000008025000000000000403800004A
:1015840000000000004B000000000000807000001C
:10159400000000000096000000000000C0DA000017
:1015A4000000000000E100000000000000C2000094
:1015B4000100000000F400000100000000E8000049
:1015C4000300000014340000040D00008206000033
:1015D40040030000A0010000CF00000067000000ED
:1015E40044000000220000007F00000030300000B2
:1015F400302C000000300000300000003062000099
:101604000000000014340000040D000082060000F5
:1016140040030000A0010000CF00000067000000AC
:101624004400000022000000307800003031000047
:1016340032330000343500003637000038390000FA
:101644004142000043440000454600002048000099
:101654007A000000467200006571000075650000A4
:101664006E63000069650000732000003C200000E8
:10167400314800007A2000006172000065200000FB
:101684006E6F00007420000073750000707000001D
:101694006F72000074650000642E000000000000FA
:1016A400436F0000756C0000646E00002774000036
:1016B400206B00006565000070200000757000005C
:1016C40000000000535000004931000000000000F9
:1016D400181C00001D0300000B1300001B00000079
:1016E400181C00001D000000314100004C53000094
:1016F4000142000050760000330000002100000089
:101704000010000000230000000F00004240000011
:101714004005000041020000000000000029000014
:101724000020000057000000205200000049000083
:1017340032430000310000000808000008080000DF
:10174400080000000000000042420000494F000071
:101754003100000052410000573100000000000039
:10176400003500003F620000610000004F430000AC
:1017740044310000000000000000000000000000F0
:020000040000FA
:1017840013C4800003007800F007B2000280210037
:1017940062407800F1CCB30081404000E8CF5000B3
:1017A40013003E000000FB000003B1001100200004
:1017B400060037006A02B90000FD2F000400400053
:1017C4000201FB00020040008100E80003814000A8
:1017D400F207B200048021006441790004CDB30013
:1017E40004424100E94F5200F2FF36006000370026
:1017F40001C3B300814F500059003A008300E80050
:10180400F107B20062C1780021C6B300814F5100D4
:1018140003003A000000EB0021002000090037001B
:1018240021C4B300814F51000F003A00F9FF370083
:10183400000040000003B1000201FB000200400070
:101844008100E80003814000F207B2000480210017
:101854006441790004CDB30004424100E14F5200D9
:10186400F3FF36004200370081C7B300814F5100B7
:1018740003003A000000EB002100200010003700B4
:1018840081C5B300814F51001E003A00F9FF3700B3
:101894004400DD00E9CF520002003E000003B10025
:1018A400040037000254A0000580210082727A00EF
:1018B4007005B1000201FB00020040008100E80055
:1018C40003824000F407B2000280210062417A00E2
:1018D40005CDB30085424100E9CF5200ECFF36004C
:1018E400F6CBB30006434100E54F5300E8FF360052
:1018F400F6C9B30006434100E54F5300E4FF360048
:101904001B003700004251000000EB0011002000D2
:10191400E94F520016003E000200FB000003B10034
:10192400060037006A02B90000FD2F0004004000E1
:101934000201FB00020040008100E8000381400036
:10194400F207B200048021006441790004CDB300A1
:1019540004424100E94F5200F2FF36000400370010
:1019640011C0B30040882100014878000000050040
:1019740012C4800082804000F107B20011C48800C4
:101984000000060012C480008200E800F107B200E3
:1019940000802100E0C1780010002000A1C3B30042
:1019A40081CF510008003A000280E800F007B2003D
:1019B40010C4880072FF070011C480008100E90090
:1019C400F107B20011C488000000060012C48000B0
:1019D4008200E800F107B20000802100E0C1780035
:1019E4000000EB00B1C3B30081CF510008003A00FE
:1019F4000280E800F007B20010C4880060FF07000E
:101A040011C480008100E900F107B20011C488000C
:101A14000000060011C480008100E800F107B20054
:101A24000080210060C1780080C7B300804F51005E
:101A340002003A0011C488001000050040C6B3003B
:101A4400804F510002003A0011C4880020000500B4
:101A540020C6B300804F510002003A0011C4880030
:101A6400300005000040EB0073C7B300834F510002
:101A740002003A0011C4880040C0B3000000060010
:101A840010C48000020037000000E800F007B20034
:101A9400018021006141780001C2B300814F5100EF
:101AA400F9FF320010C4880000000600E8874700F0
:101AB400889FBE008A9FBE008C9FBE008E1F780048
:101AC4000004BE000205BE0020912800B0530200AD
:101AD400000000000800E00004003D0060912800C0
:101AE400B0530200000000000300370008407800F3
:101AF400825202000000000080912800B0530200CE
:101B0400000000000007EB000006EB002D0037008A
:101B14000C00E000050032000C06E900B09128003A
:101B2400B053020000000000260037000E00E00061
:101B340021003200B0912800B053020000000000E0
:101B44000007EB001F0037000C00E0001A003A0009
:101B54000D40780070520200000000001E002000BA
:101B6400180037000B00E00043003A0000CDB3003A
:101B740000C04600E94F50000F003E00E30F56003E
:101B84000500340070C0B300705202000000000071
:101B94004C0020000B0037000D407800705202000A
:101BA400000000008D4078007480570001707E00B2
:101BB4000C06E8000300370070C0B3007052020046
:101BC400000000006252020000000000804678001D
:101BD400EDCF56000D00320005003C00E8CF560062
:101BE400CBFF3200EACF5600E0FF3A00070037008F
:101BF400D0C2B30080CF5600D3FF320080C7B300F9
:101C040080CF5600D9FF3A00D6FF3700F091280064
:101C140096530200000000000C00E000190032009E
:101C2400F58057000000EB00040037006A01B9009A
:101C34005100FB000003B100020040000C06E90063
:101C4400FAFF3B00890F5000060035008A0F500050
:101C540004003C000E00E000090032000004EA0029
:101C640008003700B101200080EC2000DE6502008E
:101C74000000000094FF37000084EB0001003700EF
:101C840000047800080078004F0778004F06BE0073
:101C94004F05BE004F04BE008F00B10000000600D7
:101CA4000E00FA00889FBE008A9FBE0019C48000FF
:101CB4008904E900F907B200180020002600370063
:101CC40000802100E0C07C000104E00020003A0014
:101CD4000905E800FA07B20060407D000004E00056
:101CE4001B0032000840780082520200000000000D
:101CF40000922800B0530200000000001B002000E6
:101D04000300370070520200000000008B05E80059
:101D140009804500F007B20001802100614078008D
:101D24000004E000F7FF3A00080044000A017800CC
:101D3400F6805700823078000804E800E70F54006A
:101D440008003200F09128009653020000000000C1
:101D54008904E900F907B20010C48000808F5400A0
:101D6400D7FF3A003092280096530200000000008A
:101D74007100200010742000DE65020000000000E5
:101D84001300200008017800830078000000EB00B5
:101D940046FF07008000E800E18F5000060036008F
:101DA40000004000F6805700E102780004C480007F
:101DB4000000EB0009003700F09128009653020060
:101DC40000000000100020001600370084004000CE
:101DD400F107B20003F178000000E800850040003C
:101DE400F107B20002802100E2C178000304E000A0
:101DF400F6FF3A0001C480008100E900F107B20057
:101E040011C488008180E80000804000F007B2001F
:101E140000C488000000E900F007B20003717800F4
:101E24000000EB004F05BE004F04BE000080FA0026
:101E340000000600889FBE008A9FBE0010C4800078
:101E44000000E800F007B20010C488000CFF07008F
:101E54004BFE07000000E00039003A000005EB00EB
:101E64000A40E800825202000000000000922800AC
:101E7400B0530200000000000903200009D0B9009B
:101E84008002B000088D2100080040009653020033
:101E9400000000000A05E800E40F5500F0FF3A00D6
:101EA40071012000606D2000DE650200000000006A
:101EB400408821000048EB00130020000A0178004C
:101EC4008300780003007800F8FE07000005E900AD
:101ED4000000E800E10F500003003E00E100200094
:101EE400D06E20002F00370020CF80000980B90079
:101EF4002002B0006800780000000100EA610200DE
:101F0400000000002ACF880009D0B900FE04400078
:101F140068807C0000000100509228009653020063
:101F2400000000000A00E00019003200C222A800EC
:101F3400A09328009653020000000000140037000C
:101F44000004E900E30F540014003C000A032000DD
:101F540020CF80000A80B9002002B000098D210042
:101F64006900780000000100EA610200000000003E
:101F740028CF88000AC5B9007E05450069007D00A8
:101F8400000001000800E00001003200C222A800A5
:101F9400510020005057200002003700510120005A
:101FA400C0722000DE6502000000000000C4800052
:101FB4000000E900F007B20010C488004F05BE001D
:101FC4004F04BE0000000600881F7800A097280078
:101FD400B053020000000000E0C2B30070520200DF
:101FE40000000000A09E2100104078007052020002
:101FF4000000000031CF8000F0442000808F5000AA
:1020040003003A0080982800B0530200000000004A
:10201400F09128009653020000000000F099280077
:10202400B053020000000000B0C5B30070520200BB
:10203400000000000004EB00050037000800E00089
:102044000300320000C2B30070520200000000001E
:102054000203200002C1B900818F21000100410068
:10206400B0530200000000000804E800E40F54002C
:10207400F2FF3A00D0C5B300705202000000000025
:10208400D1002000A080200098650200000000001C
:10209400A1BF2A000000EB008251020000000000F2
:1020A400000478004840DE00825202000000000074
:1020B400E0C2B30070520200000000000840780043
:1020C4008252020000000000F091280096530200A2
:1020D40000000000610020003076200098650200B6
:1020E4000000000030CF8000B65402000000000061
:1020F4007100200010EC2000986502000000000030
:1021040040CF8000B654020000000000809C2800EC
:10211400B05302000000000031CF8000F0442000E2
:10212400808F500002003A00509D280001003700C3
:10213400809D2800B05302000000000040CF8000C2
:1021440021042300810F50000E00320004003E00E1
:10215400F103B100810F500010003A00070037006E
:1021640031042300810F500008003200E380400056
:10217400810F500009003A0006003700B09D280086
:1021840007003700E09D280005003700109E280056
:1021940003003700409E280001003700709E28008D
:1021A400B053020000000000B09E280096530200C5
:1021B40000000000E101200090762000DE650200AE
:1021C400000000004F04780000000600C802B600BA
:1021D40002003200D09E280001003700009F280032
:1021E400B053040000000000CA02B600020032002E
:1021F400309F280001003700609F2800B05304007E
:1022040000000000A100200040072100DE6502005C
:102214000000000061042000C00C2100DE65020003
:1022240000000000A1012000E007210098650200E1
:10223400000000000003200021CF80000088B900C6
:102244004002B000018D210061007800000001000F
:10225400A100200080092100986502000000000010
:1022640000402000D9FF070000102000D7FF07001E
:1022740000202000D5FF070000042000D3FF070042
:1022840000082000D1FF0700F091280096530200B7
:102294000000000041002000201121009865020088
:1022A4000000000021E3A800A00020002262020038
:1022B40000000000CA5202000000000011002000CB
:1022C400B0372000986502000000000090C0B30001
:1022D4007052020000000000900020002262020000
:1022E40000000000CA52020000000000110020009B
:1022F400B0372000986502000000000090C0B300D1
:102304007052020000000000C0002000226202009F
:1023140000000000CA52020000000000110020006A
:10232400B0372000986502000000000090C0B300A0
:102334007052020000000000B0002000226202007F
:1023440000000000CA52020000000000110020003A
:10235400B0372000986502000000000090C0B30070
:10236400705202000000000021E3A9000040200098
:102374009DFF0700001020009BFF070000202000A5
:1023840099FF07000004200097FF070000082000C1
:1023940095FF0700F0912800965304000000000008
:1023A40051002000509220009865020000000000B7
:1023B400C1BF2A000000EB008251020000000000AF
:1023C400B65402000000000061002000A09220002A
:1023D4009865020000000000E1BF2A000000EB0045
:1023E4008251020000000000B65402000000000008
:1023F400F09128009653020000000000C100200064
:1024040070782000DE650200000000007DFF0700F8
:10241400C202AB000300320011012000A0622000C0
:102424000200370021012000B063200098650200FB
:1024340000000000C0C2B30070520200000000009F
:1024440000C2B3007052020000000000CB62AB0077
:102454000300320041012000705D200002003700BB
:1024640051012000205C200098650200000000005B
:10247400C0C2B300705202000000000000C2B300EA
:102484007052020000000000809C2100104078007F
:1024940070406000030032002102200030792000E7
:1024A40002003700E1012000507B2000DE650200BD
:1024B40000000000809C210010407800684060000B
:1024C40003003A00B1012000307D200002003700F3
:1024D400C1012000E07E2000986502000000000099
:1024E400C0C2B300705202000000000000C2B3007A
:1024F4007052020000000000B1012000B01A210057
:102504009865020000000000709B210010407800D4
:102514008252020000000000F0912800965302004D
:1025240000000000809C210010407800634060009F
:10253400E14F500003003A005101200000592000EF
:102544000200370061012000A0572000DE65020070
:10255400000000000003200021CF80000088B900A3
:102564006002B000018D21006100780000000100CC
:10257400C100200070782000DE6504000000000027
:1025840010C480000000E800F007B20010C4880006
:102594003BFD07007AFC07000000E900E30F500050
:1025A40002003E0010CF88000D0037004088210053
:1025B4000048EB002102200070812000DE6502004B
:1025C400000000008001EB00420020001100200008
:1025D4001000200035FD0700219E21008008E9003D
:1025E4002101200090832000DE650400000000002B
:1025F400881F780010C480000000E800F007B200D3
:1026040010C488001EFD07005DFC07000040E900BF
:10261400E94F500003003E00019E210080487800ED
:102624000D003700408821000048EB00D10820004D
:1026340060872000DE650200000000008001EB00DE
:10264400A2002000110020009000200017FD0700C8
:10265400019E21008048E9000044EB00009E210017
:1026640091C0B30090CF100010003A0004FD0700A1
:1026740043FC0700004478000004E0000B003A002B
:102684004188210080487800909F280096530200DA
:10269400000000008001EB00F2FF27008000EB0047
:1026A4002002200001FD07000044780041012000C1
:1026B40030902000DE6502000000000011012000BF
:1026C400A0192100DE65020000000000B6510200DE
:1026D400000000000004E000FCFF3200009E210026
:1026E40091C0B30090CF100003003A000840780076
:1026F4000C5502000000000096510200000000008A
:10270400625202000000000001C2B300814F500079
:10271400FBFF3A004F04780000000600E8874700FA
:10272400889FBE008A9FBE008C9FBE008E1F7800CB
:102734000000EB0010C4880000C48800409E210003
:102744000008EB00408821000048EB000000EB008B
:10275400080037000069EB008100E8000302200054
:10276400838F5000FBFF3A000000E800E30F5000A5
:10277400050032007801B9004188210001014100BF
:102784008000EB00F3FF37000000EB0070C6880008
:102794000004EB000005EB008004EB0000032000C4
:1027A40022CF80000091B900818F210001004100F7
:1027B400B05302000000000010A12800B053020032
:1027C400000000008006EB0070C680000000E000FE
:1027D4003C0032000000E90070C688008005EB0070
:1027E4000A00370001C480000280210000F1780053
:1027F40070520200000000008B05E80000C4800055
:102804000000E800F007B20000C4880070C6800031
:102814007800B900008045005188210061407800AB
:102824000004E000EFFF3A000000EB0070C68800EF
:1028340024003700809C2100104078006440600030
:10284400200032000C03200020CF80000C80B9004F
:102854007A0040000B8D21006B007800000001001D
:102864000004E0001700320020CF80000C80B90083
:102874008002B0000B004000B053020000000000D2
:1028840010A12800B0530200000000001BC4800007
:1028940000C48000808F55000A0032000600370013
:1028A4000080210060C07D00705202000000000022
:1028B400FB07B2008B05E80000C48000808F550040
:1028C400F7FF3A00BE510200000000000004E000DF
:1028D400D8FF3200125502000000000000467800C4
:1028E4000C04E00003003200185502000000000050
:1028F400B5FF3700625202000000000080457800F6
:10290400E8CF5500200032000F003E00E2CF550012
:102914008B00320005003E000B04E00092013200FF
:10292400E1CF550096013A0060013700E5CF55002C
:102934006D013200E6CF55008E003200E4CF550021
:102944008F013A0042003700EECF5500E500320017
:1029540005003E00EACF550072013200EDCF55006C
:1029640087013A006F013700FBCF55004E0032005B
:10297400F0C7B30080CF550035003200F0CF5500CA
:102984007F013A008200370010C48000800F540099
:10299400BD0132000800E90001C48000810F540029
:1029A40007003A0000047800F807B20008C4880061
:1029B400008021000C707C00B091280021003700B9
:1029C40000047800F807B20030A12800B0530200D8
:1029D40000000000880078008005EB000C00370040
:1029E4000106E8000280210062407E0000F17800C8
:1029F4000004E00001003A0000C2B300705202007B
:102A0400000000008B05E8008C007800F107B2009C
:102A140000C48000808F5000F1FF3A008100E9007B
:102A2400F107B20001C4880070A12800B05302006D
:102A3400000000000B4078008252020000000000F9
:102A4400A0A12800B0530200000000005EFF370080
:102A540000C48000800F54008B013200880078008D
:102A64008005EB000C0037000106E800028021001D
:102A740062407E0000F178000004E00001003A00AA
:102A840000C2B30070520200000000008B05E80091
:102A94008C007800F107B20000C48000808F5000E1
:102AA400F1FF3A00DDFF370062520200000000002F
:102AB400B1C5B300814F500043FF3A006252020097
:102AC4000000000011C4B300814F500030003200F8
:102AD40007003E00F0C05000814F50000C0032004F
:102AE400E3C04000814F500037FF3A000E0037002A
:102AF40031C4B300814F50001E0032007900390008
:102B04008140E800814F50002FFF3A000C0037004D
:102B14006252020000000000E1C7B300814F500080
:102B240029FF3A00E1003700625202000000000071
:102B3400E1C7B300814F500023FF3A00EA00370099
:102B4400E40F55000400340070640200000000002B
:102B54000005EB001CFF370010C48000800F5400F8
:102B6400490132000804E900F807B20030A1280046
:102B7400B4FF370000C48000800F540042013200CB
:102B84000804E800F807B200C0A12800ADFF370030
:102B940012C480008205E900FB07B20001C4800072
:102BA4008001EB00490037000480210064C07D00EF
:102BB4000004E00043003A000B00E900F007B20013
:102BC400644278000404E0003E0032008301E8001F
:102BD4008D8F51003B0036008D06E800810F5100B7
:102BE40005003A000A0037000042EB0084F1780047
:102BF4008100E900F107B20003802100828F5000B8
:102C0400F9FF3A0001C488000041EB0082F178002A
:102C140001C480000900370002802100624178006D
:102C24000204E00003003A008004E800F907B2005F
:102C3400040037000000E900F007B200810F5000E3
:102C4400F5FF3A0000A22800B05302000000000083
:102C54000003200022CF80000091B900818F210061
:102C640001004100B05302000000000010A1280040
:102C7400B053020000000000090478000A00370085
:102C84006C407C00705202000000000000C4800010
:102C940068707E000000E800F007B20000C48800FD
:102CA4000804E800F807B2000C8021008B0F5400E0
:102CB400F3FF3A0008C480000040EB0000767C007B
:102CC400040037008B05E900FB07B200818F550033
:102CD400B5FF3A0000C48000808F5500BAFE3A0068
:102CE400E900370013C480008305E900FB07B20044
:102CF40001C480000001EB004A0037000480210079
:102D040064C07D000004E00044003A000B00E900C8
:102D1400F007B200644278000404E0003F0032008F
:102D24000201E8000D02E900840F51003B003A0063
:102D340082067800818F510005003A000A003700AE
:102D44000042EB0004F178008100E900F107B200D1
:102D540002802100838F5000F9FF3A0001C48800EB
:102D64008041EB0003F1780001C4800009003700C2
:102D740002802100624178000204E00003003A006E
:102D84008004E800F907B200040037000000E900FD
:102D9400F007B200810F5000F5FF3A0000A22800AE
:102DA400B0530200000000000003200022CF800086
:102DB4000091B900818F210001004100B05302004D
:102DC4000000000010A12800B05302000000000021
:102DD400090478000A0037006C407C00705202003D
:102DE4000000000000C4800068707E000000E8005D
:102DF400F007B20000C488000804E800F807B20035
:102E04000C8021008B0F5400F3FF3A0008C48000AB
:102E14000040EB0000767C00040037008B05E900DD
:102E2400FB07B200818F5500B4FF3A0000C4800054
:102E3400808F550064FE3A00E18F560092003A00FC
:102E440000A22800B053020000000000000320008C
:102E540022CF80000091B900818F21000100410040
:102E6400B05302000000000010A12800B05302007B
:102E74000000000011C4800008C480000400370072
:102E84000041EB0002707C000804E900F807B2007E
:102E940000802100810F5400F9FF3A0008C4880023
:102EA4008040EB0001707C0046FE37001BC48000AC
:102EB4008B0F54007400320070A12800B05302003C
:102EC400000000000B005400F007B2008252020020
:102ED40000000000A0A12800B05302000000000080
:102EE40018C4800038FE37000BC480008B0F5400D8
:102EF4006500320070A12800B053020000000000F9
:102F040008805500F007B200825202000000000061
:102F140060A22800B05302000000000008C4800032
:102F240029FE370008C480008040EB0000802100A7
:102F340001707C000804E800F807B20008C48800A7
:102F4400F091280096530200000000000DC4800098
:102F54001BC48000408821000048EB000040EB00C7
:102F6400C0EF9F004C0037000A05E800F40F55003D
:102F740015FE3A00C05902000000000012FE37009E
:102F84000CC480000C00E800F007B20011C48000FB
:102F9400810F50003C003200FFCF55003A0036004C
:102FA400E0C7B30080CF550037003E00880F5600BD
:102FB4000C003A000B407800705202000000000040
:102FC40008C48000008021000B707C000804E80025
:102FD400F807B20008C488008040EB0001707C0050
:102FE400F9FD370070A12800B05302000000000072
:102FF40008005600F007B2008252020000000000F0
:1030040060A22800B0530200000000000CC480003D
:103014000D0037000C004700EE407E001140980080
:103024006E407E000004E000050032007052020091
:103034000000000080A22800B0530200000000003D
:103044000C06E900FC07B2000800E900F007B20032
:103054000E802100800F5600EEFF3A000B407800EE
:1030640070520200000000000B777C000804E800A6
:10307400F807B20000C480000000E800F007B200C6
:1030840000C48800D0FD370070C0B3007052020045
:1030940000000000CCFD370010C480000180210036
:1030A400614178000281FB008001EB00E107200010
:1030B400810F5100E08F59009D033E000260010022
:1030C4009E0337009A0337009903370098033700AB
:1030D40097033700960337009503370094033700AE
:1030E40093033700920337009403370090033700AB
:1030F4008F033700910337008D0337008C033700AB
:103104008B0337008A0337008903370088033700AD
:1031140087033700860337008503370084033700AD
:1031240083033700820337008103370080033700AD
:103134007F0337007E0337007D0337007C033700AD
:103144007E0337005E03370021023700E5003700B5
:10315400EE0037008801370076013700740337002A
:10316400FF01370072033700710337007003370023
:10317400720337001D0337002E033700090337009D
:103184005E0237005D0237005C0237005B023700E5
:103194005A023700590237005802370057023700E5
:1031A40056023700550237006103370060033700C9
:1031B400910137009E0037005D033700450037005A
:1031C400F8003700EE00370059033700610037007C
:1031D40055013700560337005503370054033700B1
:1031E40053033700520337005103370050033700AD
:1031F400600037004E0337004D0337004C0337009F
:103204006E0037004A033700490337006B0137006B
:10321400470337004603370045033700F300370000
:103224004303370042033700410337001B023700D2
:10323400E5023700270237000C033700F402370099
:103244003B033700C50037002D0037003B00370033
:103254002C013700360337002F00370031003700C8
:10326400160037001E0037003103370030033700E3
:1032740045003700200037002D03370022003700B7
:10328400460037002A0337007C0237002803370042
:1032940027033700260337001D00370006013700D7
:1032A40023033700220337002103370001023700CC
:1032B400780037000C0237007F00370078FA0700E7
:1032C4000000E0001D033A001BC480000DC4800010
:1032D4001A033700E66502000000000017033700F8
:1032E40039FB070020CF80000000E0001303320008
:1032F4002BFC070011033700CEFA07000F03370039
:10330400BBFC07000D0337009DFC07000B033700CF
:10331400BCFB070009033700F04002000000000076
:103324000603370020CF80000000E00026013200B1
:10333400903E02000000000000033700809C210042
:10334400C1CFB30010C8600061012000A057200065
:10335400F4023700819C2100114078000000A00095
:103364000014A10080487800510120000059200079
:10337400EC023700809C21001034A000C101200021
:10338400E07E2000DC003700809C21001034A10086
:10339400B1012000307D2000D700370020CF80000D
:1033A4000000E00008013200CB62A900C962A90054
:1033B40051012000205C2000CF00370020CF800086
:1033C4000000E00000013200809C210010407800E1
:1033D4007040600004003A0021022000F0E920005F
:1033E400DE65020000000000C962A800CB62A900EB
:1033F40041012000705D200098650200000000007B
:10340400F0912800965302000000000021E3A80078
:10341400B00020002262020000000000F10420003D
:10342400810F5000A2003E00D0A228009E00370069
:103434000000E800F007B20010C4880090F907000B
:10344400CFF80700000678000C007800E254020070
:103454000000000000A52800B05302000000000096
:103464000C407800825202000000000000A52800F1
:10347400B0530200000000000C40780070540200B9
:1034840000000000F09128009653020000000000A4
:10349400AA0237000000E800F007B20010C4880058
:1034A40077F90700B6F807000080FB006A630200A2
:1034B40000000000E3FF370020CF80000000E000A0
:1034C40005003A0011C0B30001407800125E02000A
:1034D4000000000099023700A1012000B05E200026
:1034E400900237005100200050602000DE65020089
:1034F40000000000B6510200000000000004E000DB
:10350400FCFF32000000FE008C02370070660200EF
:10351400000000000004E00088023200A100200046
:10352400A0602000DE6502000000000040062000CC
:103534004863020000000000EA610200000000008D
:10354400B6510200000000000004E000FCFF32005D
:1035540081BF2A00014001007802370009F9070001
:103564000006780003003700EA4302000000000070
:103574000C06E9000C00E000FBFF3A006F02370084
:1035840000F907000006780003003700D04302006A
:10359400000000000C06E9000C00E000FBFF3A000C
:1035A40066023700F7F80700000678000C003700C1
:1035B40061012000406120009865020000000000C5
:1035C4000444020000000000005502000000000056
:1035D400F091280096530200000000000C06E90058
:1035E4000C00E000F2FF3A005402370020CF8000C4
:1035F4000000E00074003200C002A900C202A8006A
:1036040021E3A8002000200048630200000000001D
:10361400A00020002262020000000000011B200024
:10362400810F500016003600900020002262020034
:1036340000000000712B2000810F500010003600A4
:1036440011012000A0622000986502000000000023
:10365400F0912800965302000000000000032000AF
:1036640021CF80000088B9000002B000018D210044
:10367400610078000000010040A528000A0037001E
:10368400C002A900C202A90060A628009653020045
:103694000000000021012000B063200098650200B2
:1036A40000000000F0912800965302000000000082
:1036B40021E3A9002102370020CF80000000E000B0
:1036C40041003200010320000180B9002002B00053
:1036D400018D210061007800000001005092280053
:1036E4009653020000000000C002A900C202A90013
:1036F40021012000B0632000986502000000000052
:1037040060FF3700F1002000C036200098650200F9
:1037140000000000306202000000000011002000E0
:10372400B0372000F4FF37003E62020000000000C2
:103734000202370093F807000006780061002000B9
:103744009065200098650200000000000C007800DD
:10375400F25202000000000021002000F065200069
:10376400DE650200000000000C0078001C6302000B
:1037740000000000F101370082F80700000678001D
:1037840061002000906520009865020000000000A0
:103794000C007800F252020000000000210020001A
:1037A40030EE2000DE650200000000000C0078000E
:1037B4004863020000000000E001370020CF8000D1
:1037C4000000E00003003A00D1012000505A20001C
:1037D400D40137002844020000000000D70137005C
:1037E400E4C3B300844F510001003A008041EB0070
:1037F4008100E8000200370013C0B300110020006C
:1038040000814000F207B200048021006441790085
:103814000204E000F2FF3A004088210003487800E7
:10382400FA8F50000200340011C0B3000148780040
:103834004E8821001004E000C0013A0010C480004A
:103844000000E800F007B20010C48800CCF70700BD
:103854000006780010C4800080007800F107B200F0
:103864000280210062C17800D1C3B300814F5100AE
:103874001B003A000C06E900E20F560035003E003A
:103884000000E800F007B20010C488007861B900B5
:1038940040882100000641008C0078000000EB0005
:1038A4008068EB000000E800F80F5000FCFF3A00CD
:1038B40010C4800003003700016E78000000E800A7
:1038C400F007B20001802100E1407800E2C3B300B8
:1038D40082CF5000F8FF3A0010C4880097013700E7
:1038E4000C00E00013003A005E8821001C00200058
:1038F4000C407800825202000000000060A82800FA
:10390400B0530200000000000E007800B053020023
:103914000000000010A128009653020000000000DF
:103924000C06E80078074700E40F5600F0FF3A0061
:10393400820137000C00E900E20F500005003E0050
:10394400F091280096530200000000007CC6880015
:103954007A01370010C0B300004F780077013700B8
:103964000000E800F007B20010C4880084F70700E4
:103974000006780042F8070011C48000F107B20085
:1039840000802100E0C0780090C2B30080CF5000D6
:1039940067013A000003200021CF80000088B900AD
:1039A4007C004000018D2100E10078000C007800CB
:1039B40001000100B3FE370024C2B30084CF5100DC
:1039C40001003A008040EB000201E80002003700E9
:1039D40011C0B3001200200080014100F307B200BF
:1039E40004802100E4C179000304E000F2FF3A00FE
:1039F40040882100014878000104E0004F013A00AA
:103A0400710020001066200098650200000000008C
:103A140020C2B300705202000000000013003700FF
:103A240011C48800705202000000000010C480001D
:103A34006C4078000000FB00819C210091407800DC
:103A4400E8C06000020032006A6302000000000067
:103A54000103200022CF80000191B900E800410059
:103A6400028D2100E28078000100010011C4800071
:103A74008100E800F107B2000C8021006CC07800DE
:103A840022C2B300824F5000E5FF3A0011C48800FF
:103A940070520200000000007AFE3700000320008C
:103AA40021CF80000088B900028D210062007800D7
:103AB400060037000003200021CF80000088B900F1
:103AC4000080E800018D2100610078000000010001
:103AD4001A0137000003200021CF80000088B900BC
:103AE40064004000F7FF37000003200021CF80006E
:103AF4000088B90066004000F2FF37007100200022
:103B04001066200098650200000000001CF7070002
:103B14000006780010C480000000E900F007B2003D
:103B240010C4880097F7070000077800A7F707007C
:103B34000000E0004E003200719B210080487800B4
:103B4400F1804000E80F5000020034001154A0003E
:103B5400470037001154A100450037000C007800DD
:103B64009062020000000000809C210002C2B300A9
:103B740090406100710050000104E00004003A002C
:103B840081C0B30090CF100004003A000A0037004F
:103B940002C1B300904F110007003200B0C3B3005C
:103BA4007052020000000000709B21001040780059
:103BB4008252020000000000809C21001040780026
:103BC40068406000040032000C0078006A63020060
:103BD40000000000000678000003200021CF8000D0
:103BE4000088B90068004000018D2100E1007800E0
:103BF4000C007800010001000001780000C2B3004D
:103C040082BF9F007052020000000000839C2100CC
:103C140001C4B30013C0600014003200610020002E
:103C240080662000F3B79F00986502000000000042
:103C3400FFB197009341780068C061000FB9970005
:103C440004003200020078006A63020000000000F1
:103C54000001780002007800906202000000000079
:103C640000C2B30070520200000000000E07E90019
:103C74000E00E000B9FF3A0002FE370061002000A8
:103C840080662000986502000000000061F70700CC
:103C9400004678003BF70700000778004BF7070061
:103CA4000000E00008003200719B21008048780089
:103CB400F1804000E80F5000020034001154A000CD
:103CC400010037001154A1000C04E0002D00320063
:103CD40010CF8000C0EF9F008C80FB00209E21004D
:103CE4000108E900270037000003200021CF8000ED
:103CF4000088B9006A004000018D2100610078004D
:103D040000000100819C210091407800E8C060001F
:103D1400020032006A6302000000000090620200A8
:103D240000000000809C210002C2B30090406100AA
:103D3400710050000104E00004003A0081C0B300A7
:103D440090CF100004003A000A00370002C1B3000B
:103D5400904F110007003200B0C3B300705202004C
:103D640000000000709B2100104078008252020085
:103D74000000000000C2B300705202000000000006
:103D84000E07E9000E00E000D7FF3A000C04E00043
:103D9400BCFD3200CFE897000180FB0010CF880003
:103DA400B8FD370081002000E0662000DE650200D7
:103DB400000000000003200021CF80000088B9002B
:103DC4006C0040003FFF3700810020006067200046
:103DD400DE650200000000000003200021CF800007
:103DE4000088B9006E00400036FF3700E100200073
:103DF400E0672000DE6502000000000000032000F0
:103E040021CF80000088B900700040002DFF3700EA
:103E1400E1002000C0682000DE6502000000000010
:103E24000003200021CF80000088B9007200400008
:103E340024FF3700C1002000D064200098650200F0
:103E4400000000000003200021CF80000088B9009A
:103E540074004000018D2100610078000000010021
:103E6400005502000000000034003700C5F60700CA
:103E740000067800D1002000A06A200098650200A6
:103E8400000000000C0078009062020000000000B6
:103E9400080037000003200021CF80000088B9000B
:103EA40076004000018D21006100780000000100CF
:103EB4000C06E9000C00E000F6FF3A0071FD370043
:103EC400B0F6070000067800A1002000706B200007
:103ED40098650200000000000E0037000003200077
:103EE40021CF80000088B90078004000018D2100B6
:103EF40061007800000001000080FB000055020012
:103F04000000000000C2B300705202000000000074
:103F14000C06E9000C00E000F0FF3A00010120006B
:103F2400A0692000DE6502000000000003003700E5
:103F340011C0B300408821000148780010C48000FB
:103F44000000E800F007B20010C488000000EB0095
:103F5400418821001104E0001200320051012000C8
:103F6400106C2000986502000000000010C480005E
:103F74008B0F500002003E0001C8B3000140400016
:103F84000B405000825202000000000040882100D3
:103F94000048EB00F0912800965302000000000056
:103FA4001000200001C4800012C48000810F510061
:103FB400020032000000E00037FC32001DC488001B
:103FC4000DC48800F5F937005752490054452000C4
:103FD400424954003A2020002A6E6500787420007B
:103FE400636C6F00636B2000285E290020776900F2
:103FF4006C6C200075736500207468006973200080
:1040040076616C0075654E006F206400657669000A
:1040140063652C002074720079202800414C410013
:10402400524D2900205345004152430048206D0061
:10403400616372006F20660069727300744144000A
:1040440044524500535320004D414300524F200039
:1040540020302E004D616300726F20006D656E008C
:10406400754D610063726F00202020002020310014
:1040740057495200452061006464720065737300FF
:104084000D0A200020202A00315749005245200003
:10409400524F4D0020434F004D4D41004E442000EF
:1040A4004D414300524F73003A0D0A002035310050
:1040B4002E52450041442000524F4D00202830002C
:1040C4007833330029202A00666F72002073690058
:1040D4006E676C0065206400657669006365200086
:1040E400627573000D0A200038352E004D415400CE
:1040F40043482000524F4D002028300078353500C9
:1041040029202A00666F6C006C6F770065642000BC
:1041140062792000363462006974200061646400AE
:1041240072657300730D0A0020323000342E530080
:104134004B49500020524F004D2028003078430056
:10414400432920002A666F006C6C6F007765640059
:104154002062790020636F006D6D61006E640D0054
:104164000A20320033362E00414C4100524D2000CB
:10417400534541005243480020283000784543000D
:10418400290D0A0020323400302E530045415200DC
:1041940043482000524F4D0020283000784630001C
:1041A40029414C0041524D002053450041524300E7
:1041B40048202800307845004329530045415200E7
:1041C40043482000283078004630290044657600B2
:1041D4006963650020494400732061007265200012
:1041E40061766100696C6100626C6500206279002F
:1041F400204D410043524F002C2073006565200080
:10420400283029002E52450041442000524F4D00D1
:104214002028300078333300293A20004D415400DF
:1042240043482000524F4D00202830007835350097
:1042340029534B0049502000524F4D002028300094
:104244007843430029556E006B6E6F00776E200033
:104254006D616300726F2C002074720079203F003E
:10426400206F720020283000292066006F72200021
:1042740068656C0070425500532052004553450058
:104284005420570061726E00696E67003A202A005C
:1042940053686F00727420006F7220006E6F2000EC
:1042A40070756C006C2D750070202A004E6F200014
:1042B4006465760069636500206465007465630065
:1042C40074656400204453003138530032302000B8
:1042D40048696700682050007265730020446900D3
:1042E40067205400686572006D4453003138420001
:1042F4003230200050726F00672052006573200036
:10430400446967002054680065726D0044533100AD
:1043140038323200204563006F6E20004469670024
:104324002054680065726D00445332003430340008
:10433400204563006F6E7200616D200074696D002A
:1043440065204300686970004453320034333100FF
:1043540020314B002045450050524F004D556E0012
:104364006B6E6F00776E200064657600696365008C
:1043740050574D0020646900736162006C656400ED
:10438400314B48007A2D34002C303000304B48003B
:104394007A205000574D46007265710075656E00B5
:1043A40063792000696E20004B487A002050720027
:1043B40065736300616C65003A505200323A440000
:1043C4007574790020637900636C650020696E0060
:1043D4002025200050574D00206163007469760049
:1043E40065455200524F52003A205000574D20006C
:1043F40061637400697665002C20670020746F0087
:1044040020646900736162006C65410055582000A6
:1044140046726500717565006E6379003A2041004B
:1044240055582000494E500055542F0048492D003E
:104434005A41550058204800494748004155580002
:10444400204C4F0057564F004C544D0045544500E6
:1044540052204D004F444500564F4C0054414700F4
:1044640045205000524F4200453A20005645720004
:10447400726F720028292000406C69006E653A0052
:1044840020407000676D730070616300653A20001E
:104494006279740065732E00546F6F00206C6F0096
:1044A4006E67210053796E00746178002065720094
:1044B400726F72004E6F200045455000524F4D0000
:1044C4004572610073696E0067646F006E65530026
:1044D400617669006E672000746F2000736C6F0052
:1044E400742049006E7661006C69640020736C006E
:1044F4006F744C006F616400696E6700206672001F
:104504006F6D2000736C6F007420450052524F0091
:10451400523A2000636F6D006D616E006420680084
:10452400617320006E6F2000656666006563740029
:104534002068650072654100434B4E0041434B00C7
:104544004932430020535400415254002042490050
:104554005449320043205300544F50002042490034
:104564005449320043206D006F6465003A0D0A001F
:1045740020312E0020536F0066747700617265004D
:104584000D0A2000322E2000486172006477610019
:1045940072655300657420007370650065643A00A9
:1045A4000D0A2000312E20007E354B00487A0D0084
:1045B4000A2032002E207E0035304B00487A0D0050
:1045C4000A2033002E207E00313030004B487A0020
:1045D4000D0A2000342E20007E343000304B480079
:1045E4007A574100524E49004E473A002048410054
:1045F400524457004152450020493200432069008B
:1046040073206200726F6B00656E20006F6E200075
:104614007468690073205000494321002028520027
:1046240045562000413329005365740020737000FF
:10463400656564003A0D0A0020312E0020313000F7
:10464400304B48007A0D0A0020322E00203430000E
:10465400304B48007A0D0A0020332E0020314D00E3
:10466400487A490032432000286D6F0064207300AB
:10467400706429003D28200020302E004D61630025
:10468400726F20006D656E00750D0A0020312E00DA
:10469400376269007420610064647200657373009A
:1046A4002073650061726300680D0A0020322E00D9
:1046B4004932430020736E006966660065725300D8
:1046C40065617200636869006E67200049324300C7
:1046D400206164006472650073732000737061006C
:1046E40063652E0020466F00756E640020646500CB
:1046F400766963006573200061743A00536E690043
:1047040066666500722842004153490043295200FD
:104714006561640079612F00412F400020636F00C0
:104724006E7472006F6C7300204155005820700045
:10473400696E61002F412F00402063006F6E74008A
:10474400726F6C007320430053207000696E430045
:104754006F6D6D00616E6400206E6F0074207500D3
:104764007365640020696E0020746800697320001A
:104774006D6F6400655075006C6C2D0075702000C1
:1047840072657300697374006F727300204F460082
:10479400465075006C6C2D007570200072657300B6
:1047A400697374006F727300204F4E0053656C0080
:1047B400662D74006573740020696E0020486900DA
:1047C4005A206D006F646500206F6E006C79520092
:1047D4004553450054424F004F544C004F41440050
:1047E4004552410055582000494E500055542F0061
:1047F40048492D005A2C200052454100443A2000DB
:10480400504F57004552200053555000504C49001A
:10481400455320004F4E50004F574500522053003F
:10482400555050004C49450053204F004646440023
:104834004154410020535400415445003A2044005F
:10484400454C4100592075007357520049544500A6
:104854003A205200454144003A2043004C4F430063
:104864004B2C200031434C004F434B002C20300094
:104874004441540041204F005554500055542C00DD
:104884002031440041544100204F550054505500FC
:10489400542C200030202A0070696E0020697300B7
:1048A400206E6F0077204800695A43004C4F430044
:1048B4004B20540049434B00533A200052454100D9
:1048C4004420420049543A00205379006E74610038
:1048D4007820650072726F0072206100742063009A
:1048E4006861720020782E002065780069742800C1
:1048F40077697400686F75007420630068616E00E6
:10490400676529006E6F20006D6F64006520630089
:1049140068616E00676523003A204E006F207300C3
:104924006F667400776172006520720065736500BC
:1049340074206F006E207600342C2000757365009F
:10494400207468006520720065736500742062003D
:10495400757474006F6E2E004E6F6E00657869007A
:10496400737465006E74200070726F00746F63005E
:104974006F6C2100782E200065786900740D0A00A0
:10498400496E7600616C690064206300686F690099
:1049940063652C00207472007920610067616900EE
:1049A4006E444500564944003A68740074703A00F5
:1049B4002F2F6400616E670065726F00757370005D
:1049C400726F74006F747900706573002E636F00EA
:1049D4006D2A2D002D2D2D002D2D2D002D2D2D007A
:1049E4002A4F7000656E200064726100696E2000B9
:1049F4006F7574007075740073202800483D48007A
:104A0400692D5A002C204C003D474E0044294E008D
:104A14006F726D00616C20006F75740070757400A6
:104A240073202800483D33002E3376002C204C00A0
:104A34003D474E0044294D005342200073657400E5
:104A44003A204D004F5354002073690067206200E0
:104A5400697420006669720073744C00534220002C
:104A6400736574003A204C00454153005420730090
:104A740069672000626974002066690072737400BB
:104A840020426F006F746C006F61640065722000D7
:104A9400762031002E20480045580D000A203200AF
:104AA4002E20440045430D000A2033002E204200EE
:104AB400494E0D000A2034002E2052004157440074
:104AC400697370006C61790020666F00726D61001B
:104AD40074207300657456006F6C74006167650020
:104AE400206D6F006E6974006F7273003A20350098
:104AF400563A2000207C2000332E3300563A200002
:104B0400207C2000565055004C4C5500503A200053
:104B14005365740020736500726961006C20700035
:104B24006F72740020737000656564003A20280079
:104B340062707300290D0A0020312E0020333000EA
:104B4400300D0A0020322E002031320030300D00AA
:104B54000A2033002E203200343030000D0A2000A9
:104B6400342E200034383000300D0A0020352E0059
:104B74002039360030300D000A2036002E20310056
:104B840039323000300D0A0020372E00203338002F
:104B9400343030000D0A2000382E2000353736001E
:104BA40030300D000A2039002E203100313532001A
:104BB40030300D000A3130002E20420052472000D0
:104BC40072617700207661006C75650041646A004B
:104BD4007573740020796F0075722000746572001B
:104BE4006D696E00616C410072652000796F75001B
:104BF4002073750072653F002043460047313A0038
:104C04002043460047323A00285C2D002F5F5C00A9
:104C14002D2928005C5F2F002D295300656C650049
:104C2400637420006F7574007075740020747900CB
:104C340070653A000D0A2000312E20004F70650087
:104C44006E206400726169006E202800483D4800AF
:104C5400692D5A002C204C003D474E0044290D007C
:104C64000A2032002E204E006F726D00616C20000D
:104C740028483D00332E3300562C20004C3D47007D
:104C84004E442900523257002028730070642000DB
:104C940068697A00293D2800202030002E4D6100EB
:104CA40063726F00206D65006E750D000A2031007F
:104CB4002E4953004F37380031362D003320410040
:104CC40054520D000A2032002E4953004F37380049
:104CD40031362D00332070006172730065206F003F
:104CE4006E6C790049534F002037380031362D005F
:104CF40033204100545220002852450053455400AB
:104D0400206F6E0020435300290D0A0052455300C2
:104D14004554200048494700482C2000434C4F008C
:104D2400434B2000544943004B2C20005245530070
:104D3400455420004C4F570049534F00203738004A
:104D440031362D003320720065706C007920280004
:104D5400757365007320630075727200656E74006C
:104D6400204C53004220730065747400696E670020
:104D7400293A200050726F00746F63006F6C3A0020
:104D840020736500726961006C33200077697200DA
:104D940065322000776972006552460055756E00D1
:104DA4006B6E6F00776E5200656164002074790049
:104DB40070653A0020746F0020656E0064766100AF
:104DC40072696100626C6500206C65006E67740036
:104DD4006844610074612000756E690074733A0060
:104DE400206E6F0020696E0064696300617469005D
:104DF4006F6E44006174610020756E006974200058
:104E04006C656E0067746800202862006974730022
:104E1400293A200043532000454E4100424C4500AE
:104E24004443530020444900534142004C4544004C
:104E340052335700202873007064200063736C00A1
:104E4400206869007A293D00282029000D0A4400C1
:104E5400697363006F6E6E006563740020616E0099
:104E64007920640065766900636573000D0A430068
:104E74006F6E6E0065637400202856007075200004
:104E8400746F20002B355600292061006E642000C9
:104E940028414400432074006F202B00332E33003C
:104EA4005629430074726C00415558004D4F44001C
:104EB40045204C0045445000554C4C0055502000B2
:104EC400485055004C4C550050204C00565245005B
:104ED40047414400432061006E64200073757000F4
:104EE400706C790035565600505533002E335600F9
:104EF40041444300427573002068690067684200BA
:104F04007573200048692D005A20300042757300E3
:104F1400204869002D5A2000314D4F00444520009F
:104F2400616E640020565200454720004C45440001
:104F340073207300686F75006C6420006265200044
:104F44006F6E2100466F75006E642000206572004C
:104F5400726F7200732E4D004F534900434C4B0047
:104F64004D4953004F435300204F4B00204641000E
:104F7400494C5300657420007370650065643A0001
:104F84000D0A2000312E200033304B00487A0D00EA
:104F94000A2032002E20310032354B00487A0D00B1
:104FA4000A2033002E20320035304B00487A0D00A1
:104FB4000A2034002E2031004D487A00436C6F00E3
:104FC400636B2000706F6C006172690074793A0041
:104FD4000D0A2000312E200049646C0065206C000D
:104FE4006F7720002A646500666175006C740D009B
:104FF4000A2032002E204900646C65002068690094
:1050040067684F007574700075742000636C6F00DE
:10501400636B200065646700653A0D000A20310067
:105024002E204900646C650020746F0020616300C9
:1050340074697600650D0A0020322E002041630059
:1050440074697600652074006F206900646C6500E3
:10505400202A640065666100756C7400496E7000F6
:105064007574200073616D00706C650020706800B9
:10507400617365003A0D0A0020312E00204D69004D
:1050840064646C0065202A006465660061756C00C8
:10509400740D0A0020322E0020456E006453500027
:1050A400492028007370640020636B007020730033
:1050B4006B652000736D7000206373006C206800C2
:1050C400697A29003D28200020302E004D616300BC
:1050D400726F20006D656E00750D0A0020312E0080
:1050E400536E690066662000435320006C6F77009E
:1050F4000D0A2000322E53006E696600662061009E
:105104006C6C20007472610066666900632D700027
:10511400202D6600202A4200797465007320640003
:10512400726F7000706564002A464100494C450066
:10513400442C20004E4F200044415400414461005F
:105144007461200062697400732061006E64200041
:1051540070617200697479003A0D0A0020312E00E2
:1051640020382C00204E4F004E4520002A64650054
:10517400666175006C7420000D0A2000322E200038
:10518400382C2000455645004E200D000A203300DF
:105194002E2038002C204F00444420000D0A20000B
:1051A400342E2000392C20004E4F4E0045537400FD
:1051B4006F70200062697400733A0D000A20310098
:1051C4002E203100202A640065666100756C74002D
:1051D4000D0A2000322E20003252650063656900FA
:1051E40076652000706F6C006172690074793A0012
:1051F4000D0A2000312E200049646C006520310026
:10520400202A640065666100756C74000D0A200034
:10521400322E200049646C00652030005541520054
:1052240054202800737064002062720067206400B8
:105234006270200073622000727870002068690038
:105244007A293D0028202000302E4D006163720031
:105254006F206D00656E75000D0A2000312E54001C
:1052640072616E007370610072656E00742062007A
:105274007269640067650D000A2032002E4C6900D3
:10528400766520006D6F6E0069746F00720D0A0000
:1052940020332E004272690064676500207769003C
:1052A40074682000666C6F00772063006F6E740072
:1052B400726F6C000A0D2000342E410075746F006B
:1052C40020426100756420004465740065637400C5
:1052D400696F6E0055415200542062007269640087
:1052E4006765520065736500742074006F20650063
:1052F40078697400526177002055410052542000AF
:10530400696E70007574550041525400204C490078
:105314005645200044495300504C4100592C20006C
:105324007D2054004F205300544F50004C495600E8
:1053340045204400495350004C4159002053540027
:105344004F5050004544570041524E00494E4700CB
:105354003A207000696E7300206E6F0074206F0035
:1053640070656E002064720061696E002028480038
:10537400695A290020524500564944003A0D0A0052
:10538400496E7600616C690064206300686F69008F
:1053940063652C00207472007920610067616900E4
:1053A4006E6D7300525320004C4F57002C20430065
:1053B4004F4D4D00414E4400204D4F004445520096
:1053C40053204800494748002C20440041544100E0
:1053D400204D4F00444541006464720065737300BE
:1053E400206F6600205043004638350037343F00B4
:1053F4005468690073206D006F6465002072650055
:10540400717569007265730020616E00206164002B
:105414006170740065724C0043442000747970001C
:10542400653A0D000A2031002E204800443434002F
:10543400373830002028750073696E0067205000EB
:10544400434638003537340020494F002065780042
:1054540070616E0064657200294C4300442028008A
:10546400747970002061640064722900203D20007A
:1054740028202000302E4D00616372006F206D00E3
:10548400656E75000D0A2000312E4C004344200047
:105494005265730065740D000A2032002E496E00B7
:1054A400697420004C4344000D0A2000332E43004D
:1054B4006C65610072204C0043440D000A203400E6
:1054C4002E43750072736F00722070006F73690051
:1054D40074696F006E206500783A28003429200032
:1054E400300D0A0020362E005772690074652000C2
:1054F4007465730074206E00756D620065727300CC
:10550400206578003A28360029203800300D0A003A
:1055140020372E005772690074652000746573008B
:1055240074206300686172006163740065727300C3
:10553400206578003A283700292038003044690073
:1055440073706C00617920006C696E0065733A00B9
:105554000D0A2000312E200031200D000A203200D7
:105564002E204D00756C740069706C0065494E0006
:10557400495443004C4541005243550052534F0097
:105584005220530045544E006F204100434B2C00E1
:105594002063680065636B002061640061707400BF
:1055A400657243004C4B09004D4F530049094300B9
:1055B40053094D0049534F0050696E0073746100E4
:1055C400746573003A474E00440933002E33560085
:1055D40009352E0030560900414443000956500055
:1055E4005509410055580900500950000950090057
:1055F40049094900092D09004F574400092D0900A4
:105604002D2D090054784400092D090052784400D6
:1056140053434C000953440041092D00092D500007
:105624004743090050474400092D09002D312E003D
:1056340028425200290932002E2852004429090028
:10564400332E28004F52290009342E0028595700C0
:10565400290935002E2847004E290900362E280036
:10566400424C290009372E002850550029093800DA
:105674002E28470052290900392E280057542900A2
:1056840009302E0028426C006B2947004E44090063
:10569400474E440009414400430935002E3056006A
:1056A40009332E0033560900565055000941550060
:1056B400580965007865630075746500203A200018
:1056C40020617500746F7200616E670065202B00A5
:1056D4004D487A00292B6B00487A290052617700E3
:1056E400207661006C75650020666F0072204200B0
:1056F40052472000284D490044493D0031323700CB
:1057040029574100524E49004E473A0020506F003D
:1057140073736900626C65002062750066666500DB
:10572400726F7600657266006C6F7700416E790067
:10573400206B6500792074006F206500786974001F
:105744005370610063652000746F2000636F6E0006
:1057540074696E0075654E00756D62006572200097
:105764006F662000626974007320720065616400D2
:105774002F777200697465003A204300533A0D0094
:105784000A2031002E204300530D0A0020322E003F
:10579400202F430053202A006465660061756C0065
:1057A40074506F0073697400696F6E0020696E0035
:1057B4002064650067726500657353006572760046
:1057C4006F20610063746900766557006169740035
:1057D400696E6700206163007469760069747900FA
:1057E4002E2E2E002A2A2000456172006C7920009A
:1057F4004578690074212A002A42610075643E00DC
:1058040031366D003A20420050204300616E6E0034
:105814006F7420006D6561007375720065203E0031
:105824002031360030303000303030002C2044003D
:105834006F6E65002E0A0D0043616C0063756C0089
:1058440061746500643A2000090A0D004573740010
:10585400696D6100746564003A20200009206200CB
:105864007073200047656E00657261006C09090061
:105874000909090050726F00746F63006F6C200097
:10588400696E740065726100637469006F6E200054
:105894002D2D2D002D2D2D002D2D2D002D2D2D00E8
:1058A4002D2D2D002D2D2D002D2D2D002D2D2D00D8
:1058B4002D2D2D002D2D2D002D2D2D002D2D2D00C8
:1058C4002D2D2D002D2D2D002D2D2D002D2D2D00B8
:1058D4002D2D2D002D2D2D002D2D2D002D2D2D00A8
:1058E4002D2D2D002D2D2D002D2D2D002D2D2D0098
:1058F4002D2D2D00203F0900546869007320680095
:10590400656C70000909090028302900094C6900F8
:10591400737420006375720072656E0074206D00EC
:10592400616372006F7320003D582F007C5809009A
:10593400436F6E007665720074732000582F7200F6
:10594400657665007273650020580900092878009F
:1059540029094D00616372006F207800207E0900E0
:1059640053656C00667465007374090009095B0073
:105974000953740061727400202309005265730096
:1059840065742000746865002042500020202000C7
:10599400090909005D095300746F7000202409008F
:1059A4004A756D00702074006F2062006F6F740080
:1059B4006C6F61006465720009097B00095374000F
:1059C4006172740020776900746820007265610058
:1059D400642026002F25090044656C0061792000AD
:1059E40031207500732F6D0073090900097D0900CA
:1059F40053746F00702061002F412F004009410053
:105A040055585000494E2000286C6F00772F4800ED
:105A1400492F5200454144002909090022616200CE
:105A24006322090053656E00642073007472690078
:105A34006E6720006209530065742000626175007E
:105A44006472610074650900090931003233200071
:105A5400632F4300094155005820610073736900A6
:105A6400676E6D00656E74002028610075782F00E4
:105A7400435329000909300078313200332064008F
:105A84002F4409004D656100737572006520410063
:105A940044432000286F6E0063652F00434F4E007F
:105AA400542E290009306200313130000953650059
:105AB4006E64200076616C007565200066094D00F7
:105AC400656173007572650020667200657175000A
:105AD400656E63007909090072095200656164000A
:105AE40020672F0053094700656E650072617400DA
:105AF40065205000574D2F0053657200766F0900E2
:105B0400092F0900434C4B002068690020680900F4
:105B1400436F6D006D616E006468690073746F009B
:105B24007279090009095C0009434C004B206C00A0
:105B34006F20690009566500727369006F6E690011
:105B44006E666F002F7374006174750073696E0064
:105B5400666F0900095E0900434C4B00207469001C
:105B6400636B20006C2F4C0009426900746F720053
:105B74006465720020286D0073622F004C5342004C
:105B8400290909002D0944004154200068692000B6
:105B94006D09430068616E00676520006D6F6400E5
:105BA40065090900095F090044415400206C6F0035
:105BB400206F090053657400206F750074707500C0
:105BC4007420740079706500090909002E094400E5
:105BD4004154200072656100642070002F50090058
:105BE40050756C006C7570002072650073697300E9
:105BF400746F7200732028006F6666002F4F4E008A
:105C04002909210009426900742072006561640059
:105C140020730900536372006970740020656E007C
:105C240067696E0065090900093A09005265700048
:105C34006561740020652E00672E2000723A3100E1
:105C440030207600095368006F772000766F6C006F
:105C540074732F00737461007465730009092E0056
:105C64000942690074732000746F2000726561003A
:105C7400642F770072697400652065002E672E001A
:105C84002030780035352E00322077002F57090058
:105C94005053550020286F0066662F004F4E290090
:105CA40009093C00783E2F003C783D00203E2F003F
:105CB4003C303E000955730065726D0061637200EB
:105CC4006F2078002F617300736967006E2078007D
:105CD4002F6C690073742000616C6C00809C21003F
:105CE4001064A00020A221001040780068406000E9
:105CF40005003200CAC2A900F0C2B300705202000B
:105D04000000000001003700CAC2A800A100200062
:105D140090AB2000DE65040000000000809C2100A0
:105D24001064A10020A221001040780068406000A7
:105D340005003200CAC2A900F0C2B30070520200CA
:105D44000000000001003700CAC2A800A100200022
:105D540090AB2000DE6504000000000020A22100BA
:105D6400104078006840600005003200CAC2A800F4
:105D7400F0C2B300705202000000000001003700BE
:105D8400CAC2A900B100200030AC2000DE650400C6
:105D940000000000881F78000102200000CA2000D3
:105DA4009865020000000000609B21001040E8009C
:105DB400825202000000000000C2B30070520200D0
:105DC4000000000028A221009840780061C0600013
:105DD400825202000000000000C2B30070520200B0
:105DE400000000001800D1006140600082520200EF
:105DF4000000000000C2B300705202000000000066
:105E0400180078004200DE00614060008252020007
:105E14000000000000C2B300705202000000000045
:105E2400180078004300DE006140600082520200E6
:105E34000000000000C2B300705202000000000025
:105E4400809C21001080FB004400DE006140600063
:105E5400825202000000000000C2B300705202002F
:105E6400000000003100200020AE200098650200F0
:105E7400000000004F04780000000600889FBE0068
:105E84008A9FBE008C1F7800420D020000000000B3
:105E9400C20B02000000000000047800420D020062
:105EA40000000000C20B02000000000000067800A1
:105EB400420D020000000000C20B020000000000BE
:105EC40080057800420D020000000000C20B0200B1
:105ED4000000000000057800420D020000000000F0
:105EE400C20B02000000000080047800420D020092
:105EF40000000000C20B0200000000008800E9005E
:105F0400E38F500003003E00619B21008848E900B4
:105F1400010037000004EB008C00E900E18F500021
:105F240007003E0021A221000C46E90061466600FC
:105F3400114178000204A1008C487100010037006F
:105F44000004EB008B00E900E18F500008003E00E4
:105F540021A221008B45E900E1C565008BC5450000
:105F6400114178000214A1008B4871000100370030
:105F74000004EB008A00E900E18F500009003E00B4
:105F840021A221000A45E9006145650022002000A4
:105F94000255DD00114178000224A1008A487100F5
:105FA400010037000004EB008900E900E18F500094
:105FB40009003E0021A221008944E900E1C46400F3
:105FC40032002000824CDD00114178000234A1002F
:105FD40089487100010037000004EB008000E900EB
:105FE400E18F500009003E00819C21006140600067
:105FF400420020000200DD00114178000244A100AB
:10600400804871000800E00062003A0040882100E6
:106014000048EB007103200000BC2000DE65020094
:10602400000000008001EB0042002000110020006D
:1060340010002000580D020000000000619B2100A8
:106044008048E9005103200070BF2000DE65020093
:10605400000000008001EB0022002000110020005D
:1060640010002000580D02000000000028A22100AA
:106074000040E90061406000984078000104A100FC
:1060840000CC700031042000C0C22000DE65020094
:10609400000000008001EB0022002000110020001D
:1060A40020002000580D0200000000000040E9001C
:1060B4006140600000404000984078000114A10055
:1060C40000CC700011032000F0C62000DE65020041
:1060D400000000008001EB002200200011002000DD
:1060E40010002000580D0200000000000040E900EC
:1060F40061406000290020000900DD00984078001C
:106104000124A10000CC7000D1012000601C2100FA
:10611400DE650200000000008001EB000901780048
:106124001100200009007800580D02000000000052
:106134000040E90061406000310020000100DD0002
:10614400984078000134A10000CC7000F1042000D4
:10615400E0932000DE650200000000008001EB00F7
:10616400090178001100200010002000580D0200E1
:1061740000000000819C210061406000420020007A
:106184000200DD00114178000244A1008048710042
:1061940001003700FFFE0700809C21001064A1006D
:1061A4004F0678004F05BE004F04BE0000000600F5
:1061B4000101200040062100DE650400000000000B
:1061C40041E2A900819C210091407800F0C0600068
:1061D40004003200CF22A800CF02A800CEC2A8003B
:1061E40003003700CF22A900CF02A900CEC2A90024
:1061F40001FE2F0043358000038160007200B3006C
:1062040042358800F30F2E004236800082816100FF
:10621400027020000301710042368800433680007A
:10622400838060000130A00041368800CAC2A80003
:10623400C8C2A900C902A900C8E2A800C922A900CD
:106244000080FB001012880042A2A80010D1800038
:10625400610160004611DD00111280000160A1009F
:106264008100710011128800C700DD000110B20026
:10627400121280000280A1000281700012128800B4
:106284004700DD000020B200111280000190A1003F
:1062940081007000111288004422EF004022EF00B8
:1062A40041E2A80000000600609B21001080FB0072
:1062B40011B7280061407800C1FF070010D18000A9
:1062C4004300DD000004B200F1FB2F0052168000F1
:1062D4008280600081007000511688000000060072
:1062E40041E2A90040358000F001B3004035880048
:1062F400F00F2E00C826B60000FE2F00C826B600F8
:10630400CF22A900CF02A900CEC2A9000000060036
:10631400F3FF37000080FB00401288008540AB008B
:10632400FEFF3200401280008540A90000000600F4
:10633400F8FF070080407800809C210003C4B3006C
:1063440010C161000000EB00010032000180FB007D
:106354000000060000C0EB00EEFF07000080FB0019
:1063640000000600C8C2A800C902A800C8E2A8002C
:10637400C922A80000FE2F00523580008200600070
:106384006100B300513588007435800084006000DA
:106394006100B300713588004535800085006000D8
:1063A4009100B30041358800F20F2E00463580007D
:1063B40086016100018020008381700043358800DC
:1063C400AC06B6007000B30060358800603580000C
:1063D400000161000281700062358800609B210029
:1063E4001080FB0011B72800614278000482FB0092
:1063F4001412880010D18000610160004611DD0094
:10640400F3FB2F001512800085806100810071006C
:10641400111288004700DD000010B200F1EF2F00D8
:1064240016128000868260008502700015128800B2
:106434004422EF004022EF0014138800141380005C
:106444008481610083017100131388001513800097
:106454008580600081007000111388006422EF00C1
:106464006022EF004822EF006822EF004322A900D7
:106474006322A9004362A80042A2A9006362A800A3
:1064840062A2A90040C2A90060C2A9004402A800F7
:106494006402A8000000060041E2A9004362A900CA
:1064A40061E2A9006362A90050358000F001B300E5
:1064B4005035880070358000F001B30070358800D5
:1064C40040358000F001B30040358800403580003D
:1064D40001F02100008070004035880060358000A4
:1064E400F001B300603588006035800000807000E2
:1064F4006035880000000600889FBE008A9FBE00A9
:106504000044780001457800C451020000000000F6
:1065140073FF070093FF07000804E00003003A003C
:1065240042E2A80062E2A80002003700E14F5400F2
:106534000A003E0041E2A80061E2A800070037001B
:106544000904E00005003A00CAC2AB0004003200AE
:10655400D0C5B3001C5202000000000019C0B300F3
:1065640040A2AB0022003A0060A2AB0020003A0037
:106574004B128000E1CF540003003A00B0C5B300D1
:106584001C520200000000000A04E0000400320073
:106594000B80FB004252020000000000060037009E
:1065A400C0C5B3001C520200000000000B4078007C
:1065B4001C52020000000000401380008044780058
:1065C4000A04E0000700320080C2B3001C5202003B
:1065D400000000000980FB0042520200000000009D
:1065E40090C2B3001C520200000000008044EB0083
:1065F40040C2AB0006003A0060C2AB0004003A009F
:1066040000202000A19E2100110060001000320033
:1066140000202000A19E21001100600002003A0029
:10662400F4510200000000004022EF006022EF005D
:106634000A04E0000400320020B52800965302004A
:1066440000000000B0FF3700C222A9000D0037008F
:10665400D251020000000000BE5102000000000000
:10666400E14F5000B6FF3A00625202000000000001
:106674000A04E0000300320030B6280096530200FA
:106684000000000084FF0700609B21001080FB00D5
:1066940011B7280061407800C9FE07004F05BE000D
:1066A4004F04BE00000006008000EB00EF0F500016
:1066B400E08F580050003E00006001000F003700DA
:1066C400120037001C0037004F0037004A00370023
:1066D40049003700480037004700370046003700BC
:1066E400450037001F003700210037002300370022
:1066F4002500370027003700290037004103200018
:1067040000CC2000DE6504000000000071002000C1
:1067140070562000DE65020000000000F100200039
:10672400B0182100DE6502000000000011C0B300B3
:106734000040EB000A003700710020007056200072
:10674400DE65020000000000F1002000B018210006
:10675400DE6502000000000011C0B30001407800B3
:1067640065FF370020A221001004A1000E003700AD
:1067740020A221001004A0000B00370020A2210059
:106784001014A1000800370020A221001014A0005A
:106794000500370020A221001024A10002003700C8
:1067A40020A221001024A00010D18000610160000B
:1067B4004611DD00111280000160A100810071000A
:1067C40011128800C700DD000110B200121280000F
:1067D4000280A10002817000121288004700DD00CF
:1067E4000020B200111280000190A100810070000D
:1067F4001112880067FD370041022000E01D2000CF
:10680400DE650200000000000000060040B628001B
:10681400B053040000000000889FBE008A9FBE00A1
:106824008C1F780011C0B300609B210001487800E0
:1068340021A22100114078000000A1000010A00056
:106844000020A10080487800809C21001044A00012
:1068540080C1B3005AFE0700ECFF07006252020039
:106864000000000051A22100804878000081FB0054
:106874004411DE0043A22100824978000281FB001A
:106884008001EB00E80F5100E08F590021013E0028
:106894000260010008003700E10037001D013700E5
:1068A4001C013700F20037001A013700F3003700EB
:1068B40018013700F70037000080FB008000EB0070
:1068C400EE0F5000E08F580012013E0000600100FE
:1068D4000E003700E0FF37001100370012003700C8
:1068E400200037001F003700680037000901370017
:1068F400080137000701370006013700050137009A
:10690400040137000A0037000F00370074FE070047
:106914004F0678004F05BE004F04BE00000006007D
:10692400CCC2A900F9003700CCC2A800F700370098
:1069340010C0B30070520200000000008040EB0061
:1069440010C0B3000500370010C0B300705202003D
:10695400000000008040EB0001407800E6FE0700E4
:10696400BEFF370062520200000000004804DD0050
:1069740062520200000000000086FB000806760058
:1069840062520200000000000044780062520200DB
:106994000000000001002100810F5600DD003E00D0
:1069A4004845DD000080FB000A0570000004EB0090
:1069B400810F550007003600D6003700E09D210006
:1069C400900444006252020000000000804C7800F1
:1069D4000804E8008C0F5400F8FF390050A221008D
:1069E40041C0B30090CF100001003A00CAC2A90010
:1069F4000004EB0004003700F0CE800060407C000F
:106A040044FE07000804E8008C0F5400FAFF390024
:106A1400100020001C630200000000000004EB00D2
:106A240006003700E09D21001006440000C0EB0082
:106A340038FE0700004E78000804E8008A0F54006E
:106A4400F8FF390050A2210041C0B30090CF1000DC
:106A540001003A00CAC2A80010C0B300705202007C
:106A6400000000000004EB0005003700F0CE8000B9
:106A740060407C0070520200000000000804E8003E
:106A84008A0F5400F9FF390074FF370010C0B300B7
:106A94007052020000000000625202000000000078
:106AA4000044780050A2210008487800E14F5400C7
:106AB4000400320095003900E24F540095003A007A
:106AC40008003700084078007052020000000000FF
:106AD4000040EB0070520200000000000840780003
:106AE4008D003700480020006055B8006252020053
:106AF4000000000051A22100804878004859DD00C0
:106B0400C851DE00830171004851DD000085FB009F
:106B14008005EB0002057500838575000804E90013
:106B2400F2FF3A006044B8000006EB006252020033
:106B34000000000051A22100804878004849DD008F
:106B4400C841DE00830171004841DD000084FB0080
:106B54008004EB0002047400838474000C06E800D3
:106B6400E40F5600F1FF3A00E10F4500E08F5D00AD
:106B740068003E00E10F4400E08F5C0065003E00C9
:106B84000800450089804D00E10F4000E08F580067
:106B940060003E0010C0B30070520200000000000C
:106BA4001B00370000C2B300DAFD07004856DE00C0
:106BB4000C407800D7FD07000A407800D5FD070097
:106BC4000040EB00D3FD07007052020000000000FB
:106BD400E10F5400E08F5C0020FF320080C2B3005C
:106BE400CCFD07000C407800CAFD07000A4078007D
:106BF400C8FD07000040EB00C6FD0700705202000C
:106C04000000000062045400E0845C000A05E8000F
:106C1400E00F5400E08F5C00E2FF3A000FFF370002
:106C24006F4060008048E80010C0B300705202005A
:106C34000000000030A221000048EB0006003700ED
:106C44006252020000000000B2FD07007052020010
:106C540000000000184CE80038A2210050A22100D6
:106C64009840780090CF5000F5FF3900FBFE3700C4
:106C7400A2680200000000002400370067406000A2
:106C840080487800619B2100804878000080FB00E8
:106C94001B00370021A22100114178000200A1004D
:106CA4000210A1000220A10082487800839C2100E8
:106CB4001344A1000080FB000028A300020032005E
:106CC4000204A000824878000018A30002003200E9
:106CD40021A221001114A0000008A3000200320028
:106CE40021A221001124A0000038A30002003A00D0
:106CF400809C21001044A000609B21001080FB00B8
:106D040091B62800614078002DFD070010C0B30043
:106D1400010037000040EB00705202000000000048
:106D2400CEFE3700881F7800B26702000000000022
:106D34000004E000170032003262AB0004003200AD
:106D44003100200040CF20009865020000000000C0
:106D54003242AB00040032003100200070CF20002A
:106D64009865020000000000AA670200000000000D
:106D7400000478003222AB000B003200F100200046
:106D8400A0CF200098650200000000003222A90074
:106D940005003700F100200090D020009865020023
:106DA400000000000004EB00080078004F047800A5
:106DB40000000600A26702000000000000000500B9
:106DC400881F780001022000F0DB20009865020093
:106DD40000000000689B21001840780082520200E5
:106DE4000000000000C2B300705202000000000066
:106DF40018407800E94F500002003A00C0118000AA
:106E0400040037000080FB000000400041AE280071
:106E140061007800F25202000000000000C2B300DA
:106E2400705202000000000010D080006340600037
:106E3400825202000000000000C2B300705202003F
:106E44000000000010D080004200DE0061406000BD
:106E5400825202000000000000C2B300705202001F
:106E64000000000010D080004300DE00614060009C
:106E7400825202000000000000C2B30070520200FF
:106E840000000000809C21001080FB004400DE0014
:106E940061406000825202000000000000C2B300A2
:106EA40070520200000000003100200020AE2000DB
:106EB40098650200000000004F04780000000600FE
:106EC4000200FA00889FBE008A9FBE00420D0200A5
:106ED40000000000C20B0200000000000001780066
:106EE4000004EB00EA0F510007003A00B2BF9F0014
:106EF400420D020000000000C20B0200000000006E
:106F0400000478003FB99700B2BF9F00420D020011
:106F140000000000C20B02000000000080057800A1
:106F2400420D020000000000C20B0200000000003D
:106F340000057800420D020000000000C20B0200B0
:106F44000000000080047800420D020000000000F0
:106F5400C20B0200000000003FB997008200E90064
:106F6400E98F500003003E00619B21008248E90044
:106F7400010037000001EB008B00E900E38F5000B3
:106F840007003E0021A021008B45E900E3C5650010
:106F9400C3CFB30091C161008BC8710001003700F9
:106FA4000001EB008A00E900E18F500009003E0077
:106FB40021A021000A45E900614565002300200065
:106FC4000355DD00914178000324A1008AC87100B3
:106FD400010037000001EB008900E900E18F500057
:106FE40009003E0021A021008944E900E1C46400B5
:106FF40033002000834CDD00914178000334A1006C
:1070040089C87100010037000001EB008000E9002D
:10701400E18F500009003E00819C21006140600026
:10702400430020000300DD00914178000344A100E7
:1070340080C871000200E00060003A00408821002E
:107044000048EB00D108200060872000DE650200C4
:10705400000000008001EB00A200200011002000CD
:1070640010002000580D0200000000000040E9005C
:10707400619B210080487800E94F50000B003A00E2
:10708400C1012000F0142100DE65020000000000B0
:107094008001EB00F2FF27001100200020022000F5
:1070A400580D020000000000C011880041052000B6
:1070B40080D1200098650200000000008001EB00F0
:1070C400420020001100200010002000580D020092
:1070D4000000000028A021000040E9006340600097
:1070E400C1CFB30098C0600000CC70001102200032
:1070F400C0D6200098650200000000008001EB006B
:10710400220020001100200010002000580D020071
:10711400000000000040E9006140600029002000F8
:107124000900DD00984078000124A10000CC700023
:1071340021032000D0D82000986502000000000040
:107144008001EB00090178001100200010002000EC
:10715400580D0200000000000040E900614060009A
:10716400310020000100DD00984078000134A100C6
:1071740000CC7000F1042000E0932000DE650200E2
:10718400000000008001EB000901780011002000DC
:1071940010002000580D020000000000819C210016
:1071A40061406000420020000200DD0011417800CF
:1071B4000244A100804871000D003700609B21004B
:1071C40091C0B30090CF100008003A006141B900AB
:1071D40000902000D1032000860602000000000079
:1071E40061015000E0815800C2118800F4FE0700DC
:1071F4004F05BE004F04BE000080FA0000000600E8
:10720400609B21001040780013D08000E94F5000AB
:107214000B003A00C0118000421ADE004319DE0060
:1072240061416100819C21009180FB00C408DE0063
:10723400E1C0600061426200E3C161000D003700FB
:10724400421ADE004319DE0061416100819C210085
:107254009180FB00C408DE00E1C060000080FB00F8
:107264000000400061426200E3C1610045AE2800B5
:1072740065007800286702000000000020A02100BB
:107284001040780063406000E34F500003003A0070
:1072940091C0B300709B210001487800846702000C
:1072A40000000000C01180002802E3000400360042
:1072B40001022000B0162100DE650200000000007B
:1072C400000006008E670400000000003222A900BE
:1072D40020A021001044A000809C21001024A000C4
:1072E400C1012000F0E62000DE650400000000007B
:1072F40020A021001044A100809C21001024A100A2
:1073040041012000B0E82000DE6504000000000018
:10731400881F78000004EB002900370020A021001A
:10732400104078007040600022003200A0A82800BD
:1073340096530200000000006100200080662000D7
:1073440098650200000000003262AB0004003200C5
:107354003100200040CF20009865020000000000AA
:107364003242AB00040032003100200070CF200014
:107374009865020000000000AA67020000000000F7
:1073840090620200000000003222AB0005003200CF
:10739400F1002000A0CF200098650200000000004A
:1073A4003222A900A0A82800965302000000000081
:1073B40002003700AA670200000000001800200045
:1073C400B2670200000000000004E000D3FF3A00AE
:1073D400080078004F04780000000600B100200087
:1073E400B00A2100DE650400000000001E21EF0049
:1073F4001021EF0080002000800888000821EF00A1
:107404000621EF001621EF001421EF00F008880098
:107414000000060011E1A9001FE1A900303480003A
:10742400F001B300303488001E21EF001021EF007A
:107434000621EF000821EF00000006000003BE0053
:1074440040AA2800110020005002BE00840F5300FF
:10745400858F5B00100031008100E900C208DD0067
:1074640040AA2800810040001101BE000200520021
:1074740083805A008100D1000080D30000004100C5
:1074840081804900800F5300818F5B000700360024
:107494000400BE00000006008100E800EF8F5000E9
:1074A400E9FF3A0001002000000005000200BE00D0
:1074B400000006000400FA00881F78008A9FBE00BE
:1074C40000047800CAE2A900C8E2A8000800E000AD
:1074D40006003A003101200020202100DE65020070
:1074E400000000000100370000000000CAE2AB0009
:1074F400020032002202AB00FBFF32006011B80030
:107504000005EB002202AB000800320030118000BD
:10751400C0FF0700E100200050212100DE650200C9
:10752400000000006055B80050003700B2BF9F0053
:10753400C3BF9F00ADFF0700CFB997003FB99700C5
:10754400CAE2AB00FEFF32001FE1A80011E1A8006F
:10755400CAE2AB00FEFF3A0011E1A9001FE1A90055
:1075640030348000F001B300303488001E21EF0075
:107574001021EF0040088000340880000A00E00079
:107584000C0032008000EB00C000DD000000200091
:1075940000004200E0804800E00F5100E08F5900F5
:1075A40003003200800F5100818F59000100360022
:1075B4000001BE000A05E800F90F5500DBFF3A00A0
:1075C400B2BF9F00C3BF9F0092FF07003FB997005F
:1075D400CFB9970000402200410F20008606020028
:1075E400000000000005BE000800E0001F003A0093
:1075F400009F240021002000800F5500818F5D0032
:1076040003003600F102200030222100150037006B
:10761400F1002000202521009865020000000000F0
:107624000A00BE00325302000000000041002000A6
:1076340000272100DE65020000000000F1002000A8
:107644001026210098650200000000000A00BE0018
:107654007AFF0700325302000000000041002000BE
:1076640000272100DE650200000000000A00BE00C1
:107674004F05BE004F0478000080FA0000000600A9
:10768400881F7800000478006140B800E40F5000BF
:10769400E08F580066003E000060010004003700DF
:1076A4000C00370040003700060037005400370054
:1076B400A1062000F0DD2000986502000000000013
:1076C4005F003700C062A900C082A800C8C2A80039
:1076D400C902A900B100200090E42000DE65020088
:1076E40000000000D100200040E52000DE6502001B
:1076F4000000000070660200000000000004E000CA
:107704004F0032003222A9003202AB0004003200E2
:107714002322AB0002003A003602F8002402F900EA
:10772400BE51020000000000E14F500006003A0084
:107734003322AB0004003A00625202000000000051
:107744000080FB00A01188003222AB0002003A0046
:107754002222AB00030032003222A9002222A90017
:10776400C222A900E30F5400E7FF3A00101680007C
:107774004400DD000010B200511680000180A10019
:10778400810070005116880051168000C308DE0085
:10779400E8806000101680000030A10000807000B6
:1077A40010168800D8FF3700E100200010E6200002
:1077B400DE65020000000000F1002000B018210086
:1077C400DE650200000000003222A9003202AB0094
:1077D400040032002322AB0002003A003602F80013
:1077E4002402F900BE51020000000000E14F5000E5
:1077F400F6FF3A0062520200000000001000370059
:107804008E670200000000000000EB0029FF070063
:107814008467020000000000C01180002802E30019
:107824000700360001022000B016210002003700D4
:1078340041022000E01D2000DE650200000000007F
:107844004F04780000000600B0A82800B0530400DC
:1078540000000000881F780022A0210092407800D8
:107864000100A100809C21001044A000404123009D
:1078740020D0880003CEB30003C960000042EB00AF
:10788400844178000441780011C0B30028670200E5
:10789400000000008467020000000000EAFF070007
:1078A400B2670200000000000004E0000B00320098
:1078B40020A02100104078007040600005003200D4
:1078C400AA670200000000007052020000000000DD
:1078D40002003700AA670200000000003222AB0059
:1078E400010032003222A900BE5102000000000053
:1078F400E14F5000EAFF3A0062520200000000002B
:1079040081A02100804878000081FB004411DE0042
:1079140073A02100824978000281FB008001EB0002
:10792400E90F5100E08F5900C1003E0002600100E0
:107934000900370060003700BD003700BC00370085
:1079440074003700BA00370075003700B8003700FC
:1079540081003700800037000080FB008000EB00CE
:10796400EF0F5000E08F5800B1003E0000600100AE
:107974000F003700C9FF3700110037001900370026
:10798400AB003700AA003700A90037001800370001
:10799400A7003700A6003700A5003700A400370071
:1079A400A3003700A2003700A10037002D003700E4
:1079B4008E670200000000004F04780000000600FB
:1079C40010C0B30070520200000000003222AB006D
:1079D400010032003222A90020A021001044A0009E
:1079E400AFFF370020A021001044A1008E00370013
:1079F40010C0B30070520200000000008E67020045
:107A04000000000062520200000000004800DD0097
:107A140020D0880010C0B3007052020000000000A3
:107A240028D0800062520200000000000080FB00A9
:107A34000000740020D0880013D08000421ADE00B9
:107A44004319DE0061416100819C21009180FB00AB
:107A5400C408DE00E1C0600061426200E3C161006D
:107A64006D00370010C0B300705202000000000027
:107A74003222A9003202AB00040032002322AB0000
:107A840002003A003602F8002402F900BE51020056
:107A940000000000E14F5000F6FF3A003322AB0033
:107AA400F4FF3A0062520200000000000080FB0074
:107AB400A0118800EFFF37006F4060008048E800A5
:107AC40010C0B300705202000000000060A021004A
:107AD4000048EB0009003700625202000000000079
:107AE4000080FB00A26702000000000010C0B30089
:107AF4007052020000000000184CE80068A0210049
:107B040080A021009840780090CF5000F2FF390007
:107B140063FF3700A2680200000000004200370043
:107B24006F40600080487800EA4F50000300360040
:107B3400A1C0B30080A021000148780080A02100EA
:107B44001080FB000000400001A92800E10078003B
:107B540021D088002300370022A021009240780021
:107B64000100A1000110A1000120A1000130A10029
:107B740001497800839C21001344A1000080FB008C
:107B84000038A300020032000114A000014978006B
:107B94000028A3000700320022A0210011D0800099
:107BA400E3C060000104A000C3CFB30092C1610030
:107BB40001C971000018A3000200320021A02100B5
:107BC4001124A0000008A3000200320021A021001B
:107BD4001134A0000048A30002003A00809C210058
:107BE4001044A0008E6702000000000013D0800043
:107BF400421ADE004319DE0061416100809C2100CD
:107C04009080FB00C408DE00E1C0600061426200B5
:107C1400E3C1610020D0800028670200000000005A
:107C2400846702000000000010C0B30001003700A8
:107C34000040EB00705202000000000018FF370003
:107C4400E30F500003003E0010A1A8001081A8001B
:107C5400E0030500FE0F500003003E0010A1A80041
:107C64001081A900A00F0500410F2000810F5000D2
:107C740004003E0010A1A9001081A800007D20008E
:107C84000000060010A1A9001081A90000E823004B
:107C9400000006001021EF001E21EF009C21EF00E0
:107CA40080CC80000000E00004003A0001FE2F00B8
:107CB400A26C20001289600016003700E0FF070064
:107CC40082CC8000110009000280D8000000E90085
:107CD4006008880091CC80000180B9004206200031
:107CE400110009000280D8008000FD0000FE2F0072
:107CF400CA06B6006001B30050368800D10C880073
:107D0400C10C880060002000E00C880011E1A8008C
:107D140020002000A0CC880000000600889FBE0040
:107D24008A9FBE008C9FBE001021EF001E21EF0031
:107D34009C21EF00A0CC8000E20F50000F003A001D
:107D440000FE2F00CA26B600C1002000E02B200050
:107D5400DE650200000000000000EB00A0CC8800FB
:107D640010C480000000E800F007B2000180210088
:107D7400614078000004E0007000320010C480000C
:107D84000000E800F007B20010C48800420D0200B1
:107D940000000000C20B0200000000008004780014
:107DA400420D020000000000C20B020000000000AF
:107DB400CF80DE0010050200000000000005BE00B8
:107DC4008900E90018002000E0F92000808F5000AD
:107DD400010036000004EB006011B8000A00BE0088
:107DE40094040200000000000000E0000A003400D7
:107DF40002002000832C24000A00BE00900402002C
:107E0400000000000000E00003003D00E10F54000A
:107E14001300320018002000408821000048EB00C5
:107E240011012000A02C2000DE65020000000000EB
:107E340011012000B02D2000986502000000000010
:107E44008001EB0002FA2000110020002003200032
:107E5400580D020000000000800478000100370083
:107E6400280020000900780075FF070011000900B0
:107E74000980D8008004E900E20F54000E003200AB
:107E840001012000902F20009865020000000000EE
:107E94008001EB00320620008000EB00200320006C
:107EA400580D020000000000CF80DE001005020023
:107EB400000000000005BE006148B800740502001F
:107EC400000000000006BE0002002000832C2400F5
:107ED4000A00BE000C040200000000000001BE0005
:107EE4000C00BE001E06020000000000DA040200BE
:107EF400000000000001BE0001FE2F00503680008B
:107F0400808060006101B30051368800D20C880083
:107F1400C20C880060002000E00C8800690888001A
:107F240011E1A800A100200090302000DE650200CD
:107F34000000000020002000A0CC88004F06BE00F6
:107F44004F05BE004F04BE00000006000EA1EF0066
:107F54000CA1EF000821EF000621EF001621EF002D
:107F64001421EF0080002000F0088800400F20005A
:107F7400E008880000402200D00888008780A9001B
:107F84001FE1A80011E1A8008780AB00FEFF3200CA
:107F940011E1A9001FE1A90031088000A1CD8800EA
:107FA400420880008001EB00C011DD0002002000C7
:107FB40002804000E080490080CD880091CD880097
:107FC400000006001E21EF001021EF00C942A800A6
:107FD40000FE2F008606B600A000B30030348800EF
:107FE400A003200080088800D8FF0700F20F2000BB
:107FF400820F5000E08F5800050036004809DD006C
:10800400C801DE00830171004801DD00040037006F
:10801400A000200080088800CCFF07000001BE00FB
:1080240031348000F101B300313488001E21EF00A7
:108034001021EF000200BE0000000600889FBE0071
:108044008A9FBE008C9FBE008001780084A0A90096
:108054008420A900F10F2E0070348000808060001D
:1080640000A02000010070007034880002FE2F0080
:108074007034800000016100A200B30072348800F3
:108084000821EF000621EF0080002000800888000E
:1080940011E1A80030002000300A880030082000D8
:1080A400100A880050CD800061CD800002003700A6
:1080B400000A80008000EB004261AB00FCFF3A0044
:1080C40050CD880061CD880001003700200A80006F
:1080D4004661AB00FDFF3A004261AB00FEFF320097
:1080E4000C0A80008006EB003CCD88004DCD880052
:1080F4002A0A80008005EB00FACC88000BCD8800AA
:108104006000B800B0CC8800C1CC880056CD800097
:1081140067CD800014CD800025CD8000D8CC8000B0
:10812400E9CC80000001EB00130037004261AB0092
:10813400FEFF3200060A80008003EB00240A800060
:108144008002EB000C0653008D865B000A0552008A
:108154008B855A00C055DD000A0020000C04450040
:108164008D844D000000440081804C000201E80031
:108174000405BE000606BE00830F5100EBFF390064
:1081840056CD880067CD88003CCD88004DCD880051
:1081940014CD880025CD8800FACC88000BCD88004A
:1081A400D8CC8800E9CC8800B0CC8800C1CC880049
:1081B40072CD88004221EF004221EF0011E1A900B5
:1081C4006119B80086060200000000004F06BE00D8
:1081D4004F05BE004F04BE0000000600889FBE008D
:1081E4008A9FBE00A0CC8000E20F500005003A0038
:1081F400F101200030312000DE65020000000000A3
:1082040058013700F1002000203320009865020057
:10821400000000001E21EF001021EF00C942A80059
:1082240000FE2F008606B600A000B300303488009C
:10823400A00320008008880044FF07000004BE005B
:108244006055B800F2FF2300820F5000E08F580001
:1082540005003600C84CDD004840DE00890470008B
:108264004844DD000D003700B1002000A0132100B8
:108274009865020000000000A0002000800888002B
:1082840032FF07000004BE006055B800F2F9200078
:10829400820F5000E08F5800040036000800BE0032
:1082A400C25302000000000026013700C0B22800BB
:1082B400E00F5400E08F5C00E00F5D00E08F5D0094
:1082C40021013200B1002000A013210098650200B2
:1082D400000000000800780058FF07006011B80093
:1082E40004A82100650020006033B8000400E10008
:1082F4000588E1000690E1000798E1004E00360091
:1083040016050200000000000001BE00703B2400BE
:10831400A13B25000C0402000000000098040200A8
:10832400000000000205BE000004BE00046A28002C
:10833400150020006033B800EA07020000000000C6
:10834400C253020000000000E0C2B30070520200F9
:1083540000000000046A2800150020006033B80003
:108364000800BE000A01BE00F80702000000000079
:108374000205BE000004BE00F070220001002000CF
:108384006011B8000040E10001C8E10002D0E10042
:1083940003D8E10024003E0000C3B3007052020081
:1083A40000000000703E2000010020006011B800B1
:1083B4000040E10001C8E10002D0E10003D8E1007F
:1083C40019003E0000C3B300705202000000000018
:1083D40030062000010020006011B8000040E100D8
:1083E40001C8E10002D0E10003D8E1000E003E0024
:1083F40000C3B3007052020000000000900020008F
:10840400010020006011B8000040E10001C8E10053
:1084140002D0E10003D8E10003003E0000C3B30032
:1084240070520200000000000800BE003253020037
:1084340000000000C3003700B4E12E001500200046
:108444006033B8000400E1000588E1000690E10013
:108454000798E1002A00360016050200000000001B
:108464000001BE00902F2000512125000C040200C1
:108474000000000098040200000000000205BE0095
:108484000004BE0004712200050020006033B8001F
:10849400EA07020000000000C253020000000000CE
:1084A400E0C2B30070520200000000000471220018
:1084B400050020006033B8000800BE000A01BE00B9
:1084C400F8070200000000000205BE000004BE0020
:1084D400703E2000010020006011B8000040E1005F
:1084E40001C8E10002D0E10003D8E10040003E00F1
:1084F40000C3B300705202000000000026003700E1
:1085040004C42900050020006033B8000400E10021
:108514000588E1000690E1000798E1003800360084
:1085240016050200000000000001BE0080B2260013
:10853400E10625000C04020000000000980402007B
:10854400000000000205BE000004BE00843E2000BE
:10855400050020006033B800EA07020000000000B4
:10856400C253020000000000E0C2B30070520200D7
:1085740000000000843E2000050020006033B800A5
:108584000800BE000A01BE00F80702000000000057
:108594000205BE000004BE003006200001002000D9
:1085A4006011B8000040E10001C8E10002D0E10020
:1085B40003D8E1000E003E0000C3B3007052020075
:1085C4000000000090002000010020006011B800AD
:1085D4000040E10001C8E10002D0E10003D8E1005D
:1085E40003003E0000C3B30070520200000000000C
:1085F40008007800F2520200000000005100370029
:1086040094162300050020006033B8000400E10044
:108614000588E1000690E1000798E1002B00360090
:1086240016050200000000000001BE0000C22B007D
:10863400E1EB24000C040200000000009804020096
:10864400000000000205BE000004BE004406200035
:10865400050020006033B800EA07020000000000B3
:10866400C253020000000000E0C2B30070520200D6
:108674000000000044062000050020006033B8001C
:108684000800BE000A01BE00F80702000000000056
:108694000205BE000004BE0090002000010020007E
:1086A4006011B8000040E10001C8E10002D0E1001F
:1086B40003D8E10003003E0000C3B300705202007F
:1086C40000000000084078001C0037001605020076
:1086D400000000000001BE000068290081D12400D0
:1086E4000C040200000000009804020000000000D6
:1086F4000205BE000004BE00A40020000500200006
:108704006033B800EA07020000000000C253020010
:1087140000000000E0C2B30070520200000000003C
:10872400A4002000050020006033B8000800BE004B
:108734000A01BE00F8070200000000008252020095
:108744000000000080B228009653020000000000E0
:1087540030348000F001B300303488001E21EF0073
:108764001021EF004F05BE004F04BE0000000600BC
:10877400809C2100104078006340600002003A00B1
:10878400C942A80001003700C8C2A800E1002000C7
:10879400103420009865040000000000809C210033
:1087A400104078006340600003003A00C942A90009
:1087B400CB42A80002003700C8C2A900CAC2A80060
:1087C40081002000F0342000DE6504000000000079
:1087D400809C2100104078006340600003003A0050
:1087E400C942A900CB42A90002003700C8C2A900AF
:1087F400CAC2A9007100200070352000DE650400A3
:1088040000000000809C210010407800634060005C
:1088140006003A00C942A800000000000000000061
:10882400501680004A00DE0005003700C8C2A800C8
:108834000000000000000000501680004600DE002A
:10884400614060000080FB0000000600889FBE00BD
:108854008A1F78001021EF001E21EF009C21EF00F9
:10886400A0CC8000E20F500010003A0010C4800039
:108874000000E800F007B2000180210061407800A8
:108884000004E00009003A0000FE2F00CA26B600EA
:10889400C1002000E02B2000DE6502000000000083
:1088A4000000EB00A0CC88005F00370010C48000FB
:1088B4000000E800F007B20010C48800420D020076
:1088C40000000000C20B02000000000041882100EB
:1088D4001104E0000B003A00CF80DE001005020016
:1088E400000000000004BE00020020004333240006
:1088F40094040200000000000045EB000000E000CA
:1089040011003400408821000048EB0031012000B0
:10891400301E2100DE650200000000008001EB0033
:10892400420B20008000EB00A0052000580D02003F
:1089340000000000CF80DE001005020000000000EF
:108944000004BE001AC0B30010A1A8001081A80042
:1089540002002C00A35524000800BE000C040200F1
:108964000000000002002400C34924001E06020087
:1089740000000000020020008327240052030200AC
:1089840000000000DA040200000000000001BE0044
:1089940001FE2F0050368000808060006101B3002A
:1089A40051368800D20C8800C20C88006000200078
:1089B400E00C8800204E20006008880011E1A80027
:1089C400C1002000601F2100DE65020000000000DD
:1089D40020002000A0CC8800E14F550012003A008E
:1089E40013002000420B20008000EB000080EB000D
:1089F400580D020000000000CF80DE0010050200C8
:108A0400000000000004BE006011B80090040200E1
:108A1400000000000000E000CBFF3D0010B528007E
:108A240096530200000000004F0578004F04BE007A
:108A340000000600C0BA2800B05304000000000083
:108A4400889FBE008044780068C0B30061C06400A1
:108A54004A5C0200000000008984FB008904D10004
:108A64000844E900F9FF3A00E05C0200000000005D
:108A74007052020000000000E05C020000000000F0
:108A840070520200000000004F04BE000000060007
:108A9400889FBE008A9FBE008C1F78000044780027
:108AA40081447800824578000CC8B3000C46640009
:108AB4006AC0B300614064004A5C02000000000028
:108AC4000884FB000804D1000A45E900F9FF3A00D4
:108AD4000C04E00006003A000980FB00685C020018
:108AE400000000000B80FB00685C02000000000036
:108AF4004F0678004F05BE004F04BE00000006007C
:108B0400889FBE008044780048C0B30010C0B30002
:108B14000908A30001003A000040EB004A5C02008F
:108B2400000000000844E900030032008984FB00CF
:108B34008904D100F5FF3700E05C0200000000006A
:108B4400E05C02000000000070520200000000001F
:108B54004F04BE0000000600889FBE008A9FBE002E
:108B64008C1F780000447800814478000246780025
:108B74008885FB00C65DDE000045EB00E34F550031
:108B84000C003A000B04E0000A00320010C0B300ED
:108B9400365C0200000000000B80FB00486302000A
:108BA400000000000040EB00365C02000000000002
:108BB400080037000884FB0010C0B3000808A300B5
:108BC40001003A000040EB004A5C02000000000093
:108BD4000804D1000A45E800E44F5500E7FF3A00D5
:108BE4000980FB00685C0200000000000C80FB00B0
:108BF400685C0200000000004F0678004F05BE00CC
:108C04004F04BE00000006000040EB004A5C020076
:108C1400000000000040EB004A5C0200000000007D
:108C24000040EB004A5C0200000000000040EB0042
:108C34004A5C0200000000000000EB00685C0200D7
:108C4400000000000000EB00685C0200000000006F
:108C54000000EB00685C040000000000889FBE0078
:108C640000047800814478000040EB004A5C020074
:108C7400000000000040EB004A5C0200000000001D
:108C84000040EB004A5C0200000000000040EB00E2
:108C94004A5C0200000000001880FB00685C0200CF
:108CA40000000000184090000080FB00685C020097
:108CB40000000000284090000080FB00685C020077
:108CC40000000000EFC4640002003700CEFF07007C
:108CD4008944E9000904E000FCFF3A004F04BE00A7
:108CE40000000600889FBE008A1F78000004BE00B2
:108CF400024578000040EB004A5C020000000000DE
:108D04000040EB004A5C0200000000000040EB0061
:108D14004A5C0200000000000040EB004A5C0200D4
:108D240000000000080078006A63020000000000F0
:108D3400685C0200000000004849DD004840DE0095
:108D440000007100C848DE006A63020000000000F1
:108D5400685C0200000000004048DE0001002000C2
:108D64006A63020000000000685C0200000000006A
:108D74006F4565000044EB0002003700A2FF0700C6
:108D84000844E8008A4F5400FCFF39004F0578007E
:108D94004F04BE0000000600881F780010C0B30016
:108DA4004A5C0200000000000040EB004A5C020044
:108DB400000000000040EB004A5C020000000000DC
:108DC4000040EB004A5C0200000000000000EB00E1
:108DD400685C020000000000E05C0200000000008B
:108DE40000047800E05C0200000000007052020001
:108DF40000000000084078007052020000000000EB
:108E040081FF070080FF07004F0478000000060080
:108E1400881F7800819C2100114078000040A00048
:108E24000034A1008048780018C0B300728050005C
:108E34000848780081C0B3000000E80001487800C9
:108E440020C0B300819D21008048780080C0EB00E1
:108E5400145B020000000000C922A900C902A90095
:108E6400C8E2A800084078002C5C02000000000062
:108E7400F0FE07006252020000000000C29D2100C3
:108E8400004978000082FB004422DE00B19D2100ED
:108E9400844878000482FB008002EB00EA0F520051
:108EA400E08F5A002F023E00046001000A003700E0
:108EB40051003700870037008D003700FE0137006E
:108EC40028023700FF01370026023700020237006C
:108ED40024023700A30037000080FB008000EB0071
:108EE400ED0F5000E08F58001E023E0000600100AC
:108EF40020023700DEFF37000B0037000D0037007B
:108F04000F003700120237000F0037002600370029
:108F1400280037002A0037002B0037002C003700C8
:108F24002F00370030003700D45B0200000000003F
:108F34000A023700B85B0200000000000702370095
:108F44000040EB0003023700809D210021C0B300E4
:108F540090CF100003003A00E05C02000000000023
:108F640003003700F00F20001A5D0200000000002B
:108F7400A19D210080487800809C21001040780049
:108F84006840600005003200A89D21001880FB00A5
:108F94006A63020000000000004C7800A09D2100DC
:108FA40010407800F0013700BE5C020000000000B1
:108FB400ED013700BA5C020000000000EA0137004E
:108FC40010C0B300470037000040EB000100370039
:108FD40010C0B300365C020000000000DF0137005F
:108FE4000040EB000100370010C0B300405C0200F9
:108FF40000000000D90137006F4060000049E8001C
:1090040010C0B3007052020000000000A09D2100B7
:109014000048EB0029003700625202000000000003
:10902400989D2100004C7800819C2100914078009B
:10903400E8C06000040032000080FB006A630200A4
:1090440000000000004C7800989D2100809D2100C4
:1090540021C0B30090CF100005003A001880FB0037
:10906400685C02000000000010C0B3000F0037006D
:109074001880FB001A5D02000000000080407800A8
:10908400004C7800809C210010407800684060000B
:10909400040032000180FB006A630200000000004B
:1090A400004C7800909D210010407800705202001E
:1090B40000000000A09D21001048E800C09D210090
:1090C400A19D21009140780090CF5000D2FF39003B
:1090D40068FF37006F4060000040E800C19D210038
:1090E40080487800945B0200000000009B01370078
:1090F4006F4060000049E80010C0B30070520200E5
:10910400000000006252020000000000B19D210036
:1091140080487800A09D21000048EB000B00370038
:10912400B89D210010C0B3001804E0000100350010
:109134000040EB004A5C0200000000001840780088
:10914400004C4000A09D21001048E800C09D210073
:10915400A19D21009140780090CF5000F0FF39008C
:109164007E01370041CAB300814F50001100320024
:1091740004003E00E4C05000814F500079013A00E1
:109184000700370051CAB300814F500081003200FC
:1091940081C0E800814F500072013A00D5003700C9
:1091A400625202000000000061A2210080487800A1
:1091B4006A01370060A2210010407800E14F50009E
:1091C40003003200E24F500066013A0023003700EA
:1091D40062520200000000000080FB006300B9003E
:1091E400B0CE88000000EB0007003700E09D2100AE
:1091F400100444006252020000000000004C780099
:1092040080CE80000000E80080CE880088CE8000F8
:10921400B0CE8000800F5400F4FF39000000EB0052
:1092240008003700F3CE8000808041002141900087
:10923400914090006340780047FE070080CE800094
:109244006300400080CE880080CE8000B1CE8000D4
:10925400810F5000F3FF39004001370062520200D1
:10926400000000000080FB004200DD00B0CE88005A
:109274000000EB0007003700E09D210010044400CB
:109284006252020000000000004C780080CE800092
:109294000000E80080CE880088CE8000B0CE800038
:1092A400800F5400F4FF39000000EB003300370056
:1092B4000040EB004A5C0200000000000040EB00AC
:1092C4004A5C0200000000000040EB004A5C02001F
:1092D400000000000040EB004A5C020000000000B7
:1092E40080CE8000F1CE8000614078000080FB00D9
:1092F400685C02000000000080CE8000F1CE800097
:1093040000804000104090000080FB00685C020078
:109314000000000080CE8000F1CE8000008040007C
:10932400204090000080FB00685C02000000000008
:1093340080CE800063004000E19D210011004000C8
:10934400904078006FC86000A09D21000048EB00A9
:10935400020037002CFE0700184CE80080CE800085
:10936400A89D2100F1CE800080804000B140900093
:1093740098CF1000F7FF39006400400080CE8800C9
:10938400B0CE800081CE8000808F5000C8FF3900AD
:10939400F200370060A2210010407800E14F500035
:1093A40003003200E24F5000B2FE3A0030003700B2
:1093B40062520200000000000080FB00B0CE880072
:1093C4006252020000000000B19D21008048780034
:1093D4000000EB0020003700B19D2100909D21008A
:1093E40011487800A09D21000048EB000E003700D2
:1093F400989D21001880FB000008A30002003200A1
:1094040010C0B300010037000040EB004A5C0200CA
:10941400000000001880FB000000D100004C780020
:10942400A09D21001048E800A09D210031C0B30098
:1094340090CF1000EEFF3600E05C02000000000058
:10944400E05C020000000000705202000000000016
:1094540080CE80000000E80080CE8800B0CE80007E
:1094640081CE8000808F5000DBFF390081FE370001
:1094740062520200000000000080FB00B0CE8800B1
:109484000000EB001500370022C0B30060B92000D3
:10949400A10B200013FE07003FFE070022C0B3000B
:1094A40060BB2D00A10B20000EFE070022C0B300FC
:1094B400603D2D00A10B20000AFE070036FE0700C8
:1094C40022C0B30060BB2000A10B200005FE0700F2
:1094D40031FE070080CE80000000E80080CE8800C6
:1094E400B0CE800081CE8000808F5000E6FF39002E
:1094F40060FE370062520200000000000080FB00A2
:10950400A0CE880062520200000000000080FB0030
:1095140090CE880061A2210091407800E2CF5000F3
:1095240004003A00A2CE80006511B9000200400098
:1095340008003700E1CF500002003200E3CF5000B2
:1095440088003A00A1CE80008180400001004000E4
:1095540000004000B0CE88000000EB000700370098
:10956400E09D21001004440062520200000000004B
:10957400004C780080CE80000000E80080CE880097
:1095840088CE8000B0CE8000800F5400F4FF3900F4
:1095940090CE80000000E0000300320010C0B30051
:1095A40070520200000000000000EB003900370098
:1095B400F0CE800060C17800E14F51001E003A00F7
:1095C40062A2210012417800E34F510006003A00E4
:1095D4000100400030419000A040900010409000F5
:1095E4002BFD070007003700E14F510008003A0047
:1095F4000100400030419000A040900010409000D5
:1096040055FD070080CE8000640040002100370033
:10961400E24F510020003A00010140008100E800BF
:1096240001004000C24090008CFD070080CE800005
:109634006500400017003700E24F510016003A0061
:1096440062A2210012417800E34F510004003A0065
:109654000100400010409000F9FC070005003700AD
:10966400E14F510006003A00010040001040900014
:1096740023FD070080CE80000080E800050037004D
:10968400E24F510004003A00C3FD070080CE800081
:109694000000E80080CE880081CE8000B0CE80003B
:1096A400808F5000C2FF390090CE80000000E0009F
:1096B400F0FD3A0029003700A26802000000000013
:1096C40026003700E340600001497800609B2100D8
:1096D400014878001A003700829C210092407800EB
:1096E4000140A100014978000080FB000038A3007C
:1096F40002003A000144A00001497800819D210044
:1097040022C0B300824878000028A300020032007F
:1097140032C0B30082487800829C210092407800D5
:109724000130A100014978000018A30002003200B2
:109734000134A00001497800609B2100904078002A
:10974400809D210010407800145B0200000000009E
:1097540010C0B3002C5C02000000000010C0B30075
:10976400010037000040EB007052020000000000CE
:10977400C0FD37004F04780000000600E0A121007E
:10978400104078000018A300110032000008A30064
:1097940003003A000040EB004A5C020000000000B5
:1097A40000C2B3007052020000000000310020002B
:1097B40030412000986502000000000000C2B300A0
:1097C4007052020000000000E0A121001014A1006A
:1097D400E0A1210010407800E14060000040EB006F
:1097E40002003A00E05C020000000000E1A1210058
:1097F4001114A0000080FB0000000600889FBE003A
:1098040000047800E9A121009940780062C060005A
:109814001100320000C2B3007052020000000000C8
:109824003100200030412000986502000000000053
:1098340000C2B30070520200000000009944780096
:1098440061C0640002003A004A5C020000000000AB
:10985400E0A121001014A100E0A121001040780033
:109864006140600006003A0008007800685C02006D
:1098740000000000BE5C0200000000000084FB0049
:1098840000C2B30070520200000000000800E000B3
:1098940006003A00310020003041200098650200A3
:1098A40000000000003020000500370041002000C7
:1098B40060412000986502000000000000102000B4
:1098C4004F04BE0000000600881F7800E8A12100B4
:1098D4009840780062C060000F0032004100200010
:1098E40060412000986502000000000000B92800D3
:1098F40096530200000000001844780061406400A0
:1099040003003A0010C0B3004A5C020000000000EB
:10991400E0A121001014A100E0A121001040780072
:10992400614060000F003A00D45B020000000000B8
:109934000000E0000B00320091002000C020200055
:109944009865020000000000510120005021200011
:10995400986502000000000000B928009653020038
:1099640000000000D1002000A0412000DE650200BC
:10997400000000004F04780000000600881F7800F3
:10998400E8A121009840780062C060000F00320016
:1099940041002000604120009865020000000000A2
:1099A40000B9280096530200000000001844780013
:1099B4006140640003003A0010C0B3004A5C020036
:1099C40000000000E0A121001014A100E0A121008A
:1099D400104078006140600002003A00B85B020069
:1099E40000000000C100200070422000DE6502007B
:1099F400000000004F047800000006000101200070
:109A0400404F200098650200000000000040EB0079
:109A1400825202000000000000C2B3007052020033
:109A240000000000609B2100104078008252020078
:109A34000000000000C2B3007052020000000000E9
:109A440010B928009653040000000000881F780015
:109A5400E8A121001804A100420D0200000000004A
:109A6400C20B0200000000008000E900E38F5000F8
:109A740011003E00619B21008048E90041CF800035
:109A840030002300808F500004003E00510320006A
:109A9400304920009865020000000000D7FF07004D
:109AA400E0A121001014A100809C21001044A0001A
:109AB4004F04780000000600408821000048EB00B5
:109AC4001804A100B103200080452000DE650200D7
:109AD400000000008001EB00420020001100200083
:109AE40010002000580D020000000000619B2100BE
:109AF4008048E900ECFF3700E0A121001040780025
:109B04006140600009003A00C922A800C902A80007
:109B1400CB02A900CB22A900609B210090407800D1
:109B240020C0B300145B0200000000000000060027
:109B3400E1A12100114078000010A10080487800C4
:109B44000008A3000100320007E2A900000006009B
:109B5400B1002000600B2100DE650400000000005D
:109B6400889FBE008A9FBE008C9FBE008E1F780017
:109B740000477800C451020000000000C922A80078
:109B8400C902A800CB02A900CB22A90062A0A800A8
:109B940062C0A8008660A90059168000C94CDE0086
:109BA400581680004844DE0061446400E1C4640047
:109BB4000046EB008C4578008C467800080037009E
:109BC400004478008A447800050037008A4478000D
:109BD4000044EB000200370019C0B30009447800C8
:109BE4008660AB000D003A00D25102000000000074
:109BF400BE510200000000000004E000F8FF320043
:109C0400625202000000000062A0A90062C0A90024
:109C14000E04E0004F0032004B0037008660A900BC
:109C24005A1680004955DE006145650050168000D3
:109C34004800DE00614060000D04E00028003200AE
:109C44000804E00028003A000004E000DDFF3200D0
:109C5400E7CF550008003E000C4646000A04E00029
:109C6400010032000C04A0008B45E8008A4478000F
:109C740018C0B300DAFF37000E04E000040032001D
:109C84000C80FB0042520200000000000600370076
:109C9400C0C5B3001C520200000000000C40780054
:109CA4001C520200000000000A04E000060032001A
:109CB400D0C2B3001C520200000000008045EB003B
:109CC40018C0B3001E003700B0C2B3001C5202001B
:109CD400000000008045EB0018C0B3000E00370000
:109CE4000804E000B6FF32000004E000B7FF3200D1
:109CF4000904E0000A0032000A04E000B6FF3A005A
:109D0400B0C5B3001C520200000000008045EB0007
:109D14001DC0B3000D4478008B447800B0FF3700B9
:109D240018C0B3000A04E000ADFF3200D0C5B30090
:109D34001C520200000000008045EB008B467800B6
:109D440088447800A6FF370000B928009653020023
:109D5400000000004F0778004F06BE004F05BE000C
:109D64004F04BE0000000600889FBE000004780077
:109D7400E10F54000900320003003900E20F5400DF
:109D840066003A005500370051032000405020007F
:109D94009865020000000000640037008040EB007A
:109DA40000302000705B020000000000E10220008F
:109DB40090532000DE65020000000000CB02AB00DF
:109DC400030032008004EB00CB22AB0009003A0010
:109DD40091002000C02020009865020000000000CF
:109DE400510120005021200098650200000000006D
:109DF40036003700E0A12100104078006140600087
:109E040008003A00D45B020000000000090078005A
:109E1400685C020000000000BE5C0200000000005C
:109E24000084FB000800E0001E003A0009007800EE
:109E3400906202000000000080C2B3007052020071
:109E4400000000000980D1009062020000000000C0
:109E540030B928000908A3000A003200E0A121005B
:109E6400104078006140600005003A00E05C0200A8
:109E74000000000010C0B3004A5C020000000000B3
:109E840060B92800B05302000000000010B9280097
:109E9400B05302000000000000C2B3007052020080
:109EA40000000000E0A12100104078006140600043
:109EB40002003A00B85B0200000000008904E800D8
:109EC40000102000808F5400CAFF3A0000B9280017
:109ED400965302000000000014003700E0A12100A6
:109EE40010407800614060000100320007E2A900E0
:109EF4007100200070562000DE65020000000000A2
:109F0400F1002000B0182100DE650200000000000E
:109F140010C0B30012FF0700040037004102200004
:109F2400E01D2000DE650200000000004F04BE00BA
:109F34000000060090B92800B0530400000000009F
:109F4400889FBE008A9FBE00C922A800C902A8003B
:109F5400CB02A900CB22A900C8C2A900819C210080
:109F6400114078000040A0000034A100804878002F
:109F740080C0EB0020C0B300145B020000000000AE
:109F8400ECFF0700625202000000000012A2210050
:109F9400004978008081FB00C419DE0004A221007E
:109FA400034A7800E1CF5100AC00320005003900CB
:109FB400E4CF5100C7003200E6CF5100C9003A0097
:109FC400BE0037000080FB008000EB00EF0F500064
:109FD400E08F5800C3003E0000600100C500370058
:109FE400E7FF37000D0037000F003700110037007E
:109FF400BC0037001200370013003700160037008A
:10A0040063003700B7003700B6003700B5003700EB
:10A01400B4003700B30037008D003700D45B020072
:10A0240000000000AD003700B85B02000000000033
:10A03400AA003700E05C020000000000AA0037001C
:10A044000040EB000100370010C0B3004A5C02007E
:10A0540000000000A100370062520200000000006E
:10A064004804DD0062520200000000000085FB008D
:10A0740008057500625202000000000000447800E8
:10A08400625202000000000001002100810F55000F
:10A0940094003E00C844DD000080FB008904700089
:10A0A4000004EB00818F5400070036008D00370058
:10A0B400E09D21009005440062520200000000006F
:10A0C400804D78000804E8008A0F5400F8FF390036
:10A0D400D45B0200000000000004EB000A0037001B
:10A0E400F0CE800060407C000080FB00685C0200D1
:10A0F40000000000BE5C020000000000E14F5000C0
:10A10400780032000804E8008A0F5400F4FF390094
:10A114000905E9000004EB000C003700E09D210074
:10A1240090054400E05C020000000000804D7800CF
:10A134000040EB008A0F54000100390010C0B30046
:10A144004A5C0200000000000804E800890F540083
:10A15400F2FF3900B85B02000000000010C0B30039
:10A1640070520200000000000004EB0005003700FC
:10A17400F0CE800060407C007052020000000000BD
:10A184000804E800890F5400F9FF39007DFF370007
:10A1940010C0B30070520200000000002202AB00A5
:10A1A400FEFF3200311180000140780012A221002C
:10A1B40001497800E2CF50001400320005003E004F
:10A1C4000104E0000B003200E1CF50001E003A0011
:10A1D4000B003700F0CF50001200320001C2B30070
:10A1E400814F500013003200E34F500016003A0034
:10A1F40009003700EA4302000000000012003700A3
:10A20400D0430200000000000F003700BA430200F0
:10A21400000000000C0037000444020000000000AD
:10A2240031003700809C2100C1CFB30010C860000A
:10A2340005003700819C2100114078000000A00037
:10A244000014A10080487800100020002600370088
:10A254000040EB0042FE0700200037006F40600022
:10A264000049E8000340780070520200000000003A
:10A27400F0A121000048EB000A00370062520200FE
:10A28400000000000080FB00685C02000000000089
:10A29400BE5C0200000000007052020000000000DA
:10A2A400184CE800F8A1210010A221009840780081
:10A2B40090CF5000F1FF390032FF3700E3406000D7
:10A2C4000149780020C0B300145B020000000000C4
:10A2D40002003700A26802000000000010C0B300B2
:10A2E400010037000040EB00705202000000000043
:10A2F40024FF37004F05BE004F04BE0000000600D7
:10A30400220320001241780032E0B7001180BA0025
:10A314009100BA0023032000824978004800DD0040
:10A324000080700000000600009E210010407800AC
:10A33400E94F5000050032000080FB00000040009F
:10A3440041B02800E1007800411188002022EF008C
:10A354002062A8002222EF0021E2A8002342A800E4
:10A364008560A90000000600101180004800DE008E
:10A374006140600000000600101180006140600030
:10A38400000006000000EB00C0D088001000200090
:10A39400B0D08800A09E21001090A100000006000B
:10A3A4002322AB000E003A00C0D080000000E80079
:10A3B40001002100810F500001003A000000EB0071
:10A3C400B1D08000810F500005003200C0D0880059
:10A3D400F1CE8000614078000080FB0020118800ED
:10A3E40000000600B4D08000F3CE8000C1D080000D
:10A3F4000101E8000000EB0005002100850F510079
:10A404000100320002007800840F5000070032007F
:10A414002322AB00F7FF3A00E34078008180FB0081
:10A424002111880080007800F1FF3700C1D0880036
:10A4340000000600B1D08000C2D08000828F50009E
:10A4440005003A00C222A90050CF80000090A0006D
:10A4540050CF880000000600F2CE800000F17800A2
:10A464008100E800B1D0880000002100808F5000F6
:10A4740002003A000000EB00B0D0880000000600A3
:10A48400889FBE008004780000C3B300E9FF070082
:10A4940080C7B300E7FF07004448DE006F00600098
:10A4A40088B1280068407800E2FF0700EF84640068
:10A4B40068C07C00DFFF07004F04BE0000000600F8
:10A4C4002202AB00FEFF32003011800000000600C3
:10A4D4002302AB00FEFF3200000006000110200042
:10A4E400A29E21009280600004003A002322AB0067
:10A4F400FEFF3A000000FB00201188000000060067
:10A50400889FBE008A9FBE00004478002AC0B30022
:10A514008041EB0049C6B3008885FB000981FB003C
:10A52400110009008285D800800578000304E0004A
:10A5340002003A000B04E0000700320001C3B3003C
:10A5440001C04500E5FF07000980FB000B80B9004E
:10A554000044540013C0B3000A45E9000600320069
:10A564008984FB00A2002000110009008284D80025
:10A5740080047800E8FF370001C3B30001404400C1
:10A58400D6FF07004F05BE004F04BE0000000600C2
:10A59400881F78007D02B900D30220001100090051
:10A5A4000382D80042062000110009000280D8006E
:10A5B40001047800D2FF0700E0C2B300C7FF070020
:10A5C400E94F540002003E0000C3B300C3FF07007C
:10A5D40008407800CAFF07004F0478000000060016
:10A5E400889FBE008A9FBE00800478004AC0B300E2
:10A5F4008041EB0008712200110009008884D80012
:10A60400800578000304E00002003A000B00E0003B
:10A614000600320001C3B30001C04500AFFF0700CC
:10A6240008D8B9008084540013C0B3000A45E90077
:10A6340005003200A2002000110009000284D800A5
:10A6440000047800ECFF370001C3B30001C04400EC
:10A65400A2FF07004F05BE004F04BE000000060025
:10A664000400FA00889FBE008A9FBE008C9FBE0033
:10A674000004BE008CC0B3008046EB000A102E001C
:10A684005B5F20000A01BE000800BE0086060200CF
:10A69400000000000002BE000D04E00003003A00C8
:10A6A400E00F5000E08F58000E00320001C3B300E9
:10A6B4000140420084BF9F0095BF9F0087FF0700B1
:10A6C4000A01BE000FBA97009FBA97000400BE00AB
:10A6D400AC060200000000000004540081845C0009
:10A6E4001DC0B3000C46E90007003200A2002000A0
:10A6F400030020000A00BE008606020000000000DD
:10A704000005BE00DFFF370001C3B3000140440071
:10A7140072FF07004F06BE004F05BE004F04BE0087
:10A724000080FA0000000600881F7800000478000A
:10A734000100370069FF0700384078000004E0009A
:10A74400FCFF3A00D0C0B30064FF0700A0C0B30010
:10A7540062FF07004F04780000000600881F78009D
:10A7640000047800010037005CFF070038407800DF
:10A774000004E000FCFF3A004F04780000000600EB
:10A78400889FBE008A1F78008C9FBE000004BE0014
:10A79400F0232400F1002000800F5400818F5C001E
:10A7A4001600360002242400F30020000800BE0036
:10A7B400860602000000000089FF0700C0C2B30043
:10A7C40046FF070002242400F30020000800BE0016
:10A7D400A6060200000000000004BE001A002000CB
:10A7E400703E2000800F5400E08F5C0008003E00A3
:10A7F40080AF2800D9FF0700240037000005EB00D4
:10A80400703E2000800F5400E08F5C001F00360073
:10A81400823E2000030020000800BE0086060200DD
:10A82400000000000006BE0030062000800F560025
:10A83400E08F5E000A003E000A00E00008003200DB
:10A84400E90F5600E08F5E000300360000C3B3003A
:10A8540022FF070002003700D0AF2800BFFF070027
:10A864000C0078005EFF0700C0C2B3001BFF0700A6
:10A87400823E2000030020000800BE00A60602005D
:10A88400000000000004BE001A0020003006200072
:10A89400800F5400E08F5C000A003E000A00E000D4
:10A8A40008003200E90F5400E08F5C00030036001A
:10A8B40000C3B30009FF070002003700D0AF28002F
:10A8C400A6FF07000800780045FF07004F06BE00FA
:10A8D4004F0578004F04BE0000000600889FBE00AC
:10A8E4008A1F78000045780000B028009BFF07000D
:10A8F40089C0B30008C8B3000A40640002003200F3
:10A9040010C3B3000100370000C3B300F3FE070017
:10A914008944E900030032000884FB000804D100E4
:10A92400F5FF37004F0578004F04BE000000060015
:10A93400889FBE008A1F7800010578008004780093
:10A944000004EB000300370039407800E3FE070001
:10A954000804E8008A0F5400FBFF39004F05780013
:10A964004F04BE0000000600889FBE00000478006B
:10A974002100200060B12800EDFF07004C40DE00FC
:10A9840089B1280069407800D4FE07004840DE0001
:10A994006F00600069407800D0FE07004440DE008C
:10A9A4006F00600069407800CCFE07006F0464000B
:10A9B40069407C00C9FE07004F04BE000000060089
:10A9C400889FBE00000478002100200060B12800A8
:10A9D400D7FF07004440DE006F00600089B1280003
:10A9E40069407800BDFE07006F04640069407C0084
:10A9F400BAFE07004F04BE00000006000000E0009D
:10AA04000200320010C3B3000100370000C3B300DA
:10AA1400B2FE37000080FB004011880000000600F1
:10AA24002202D50061406000000006002222A90035
:10AA3400000006009580AB000C003A00A0CF800017
:10AA4400B1CF8000808F5000080032002322AB0079
:10AA5400FEFF3A008580A9009580A80091CF800070
:10AA6400614078000080FB0020118800000006008F
:10AA7400809FBE00821F78003211800080CF80004A
:10AA840061CF80008270780080CF80000000E800F1
:10AA940080CF880071CF8000810F500001003A0000
:10AAA4009560A9008560A9004F0178004F00BE00A1
:10AAB40000400600809FBE00A0CF80000000E80098
:10AAC400A0CF8800B1CF8000810F500002003A006F
:10AAD4009580A9000400370091CF80006140780080
:10AAE4000080FB00201188008580A9004F00BE0073
:10AAF40000400600C8E2A800C902A900C922A900B2
:10AB0400C8C2A900CAE2A900CB02A900CB22A900AD
:10AB1400CAC2A90000000600501680004700DE00EB
:10AB2400614060000000060051D08000C208DE00D1
:10AB3400E1C06000014178000204A20061016100EB
:10AB44004911DD00F0DF2F0044168000840160000D
:10AB54008301710043168800E1806000C908DD00AC
:10AB6400CA02B60000807000501688004001200020
:10AB74001C63040000000000CB22A900C922A90024
:10AB8400400120001C6304000000000051D080003C
:10AB9400C208DE00E1C06000014178000204A200A6
:10ABA400610161004811DD00F0EF2F0044168000C0
:10ABB400840160008301710043168800E180600015
:10ABC400C808DD00CA02B600008070005016880074
:10ABD400400620001C63040000000000CB02A90012
:10ABE400C902A900400620001C6304000000000004
:10ABF400889FBE00804478000044EB0003003700C7
:10AC0400E2FF0700F5FF07000844E800894F5400FD
:10AC1400FBFF39004F04BE0000000600881F7800C7
:10AC2400DAFF0700581680004744DE0061446400E0
:10AC3400EAFF0700084078004F047800000006008F
:10AC4400881F78000004E00002003A00CAFF0700F1
:10AC540001003700B4FF0700CCFF0700581680003E
:10AC64004744DE0061446400DCFF070008407800CC
:10AC74004F04780000000600889FBE00D7FF07003D
:10AC8400A8A021009840780068C060000500320048
:10AC940050D080004400DE0061406000E8FF0700FF
:10ACA4001834A10089C0B3000044EB00B7FF0700CB
:10ACB4000884FB000804D100CAE2AB0002003200A1
:10ACC40000C8B30000444400C4FF07008944E900FD
:10ACD400F6FF3A00084078004F04BE00000006006A
:10ACE400889FBE008A1F780000447800BBFF0700DD
:10ACF400A9A021009940780068C0600005003200D6
:10AD040050D080004400DE0061406000CCFF0700AA
:10AD14001934A1008044EB00094578000808A30019
:10AD240002003A0094FF0700010037007EFF07008D
:10AD340096FF07000884FB000804D1008984FB0007
:10AD44008904D100CAE2AB000200320000C8B3009B
:10AD540080C44400A1FF0700A0A021001041780096
:10AD6400E3406100E2CF50000B003A00E64F55008B
:10AD740009003A00824078000130A0000808A300CE
:10AD840002003A000144A100010037000144A00080
:10AD940001487800030037000A45E800E84F5500F1
:10ADA400DEFF3A00094078004F0578004F04BE00EA
:10ADB4000000060051D08000C208DE00E1C060003F
:10ADC400014178000204A200610161004611DD0026
:10ADD400F0FB2F00441680008401600083017100A1
:10ADE40043168800E1806000C608DD00CA02B60090
:10ADF4000080700050168800400120001C6304008D
:10AE040000000000CAC2A900C8C2A9004001200075
:10AE14001C63040000000000E6FF0700A0C0B300AC
:10AE240073FF0700F7FF0700A0A02100C1CFB30004
:10AE340010C8600000000600881F780000447800F5
:10AE4400E24F540010003200E34F5400040032007B
:10AE54000804E00017003A00EFFF07001500370070
:10AE6400D4FF070010C0B30061FF0700E5FF07002F
:10AE740020C0B3005EFF0700A0A02100904078002E
:10AE840063C870000B003700CAFF07000840780051
:10AE940057FF0700DBFF07000840780054FF070056
:10AEA400A1A02100114078000000A1000014A0001E
:10AEB400804878004F04780000000600881F78005E
:10AEC400A8A0210050D0800063006000E20F500071
:10AED40005003200E30F500019003200E10F50006A
:10AEE4001A003A0020003700184078000038A30008
:10AEF400070032000048A300020032000AFF0700E6
:10AF0400010037001CFF0700A0A021001034A1009D
:10AF1400A8FF070020C0B30035FF0700B9FF0700F2
:10AF240010C0B30032FF0700A1A021001140780037
:10AF34000000A0000014A100804878000A00370037
:10AF44009CFF070020C0B30029FF0700ADFF0700E6
:10AF540010C0B30026FF0700184078000000A000CE
:10AF64000014A100004C78004F0478000000060093
:10AF7400881F7800DFFE0700A0A0210010417800A0
:10AF84000224A00071CEB3000148610062520200A5
:10AF94000000000000447800E0A021000848780088
:10AFA400E14F540003003200E24F5400F7FF3A002F
:10AFB4000200370098FF07003700370096FF0700AC
:10AFC400D9FE0700BDFF0700084078009AFF07007C
:10AFD40000C0EB0006FF070000C0EB0004FF070001
:10AFE400B6FF070030C0B30093FF07000000EB007A
:10AFF40060D088000600370060D080000000E800C0
:10B0040060D08800910F2000810F500003003600AB
:10B0140002FF07000004E000F7FF3200A7FF07006B
:10B024007DFF0700A5FF070030C0B30082FF0700C3
:10B034002000200061D080000008DD007052020072
:10B0440000000000F0A021000048EB000D003700D4
:10B0540009FF0700705202000000000006FF07000D
:10B06400705202000000000003FF0700705202004B
:10B074000000000000FF0700705202000000000002
:10B08400184CE800F8A021009880FB0060D08000F4
:10B09400808F5000EEFF390088FF0700BBFF3700A8
:10B0A40060BA2800B053040000000000625204009B
:10B0B40000000000881F7800004478000880FB002E
:10B0C4004401DE00610161004A11DD004116800087
:10B0D40001A0A1008100710041168800C600DD00B6
:10B0E4000120B200421680000290A100028170008B
:10B0F40042168800C600DD000110B200421680002E
:10B104000280A1000281700042168800C600DD00A2
:10B114000108B200421680000270A1000281700092
:10B1240042168800610060004600DD004116800080
:10B134000160A100810070004116880050002000C9
:10B144001C6302000000000000CEB3000040640055
:10B15400CB42AB00010032000044A000CB22AB0084
:10B16400010032000034A000CB02AB000100320029
:10B174000024A000CAE2AB00010032000014A000C9
:10B18400CAC2AB00010032000004A0004F047800E2
:10B1940000000600881F7800004478000880FB0047
:10B1A4000068A30003003200C002A900C202A80084
:10B1B40002003700C002A900C202A9000058A3007F
:10B1C40003003200C962A800CB62A9000200370064
:10B1D400CB62A900C962A9004401DE0061016100DB
:10B1E4004A11DD005116800001A0A1008100710008
:10B1F40051168800C600DD000120B20052168000FE
:10B204000290A1000281700052168800C600DD0081
:10B214000110B200521680000280A1000281700069
:10B2240052168800C600DD000108B20052168000E4
:10B234000270A10002817000521688006100600053
:10B244004600DD00511680000160A10081007000FD
:10B2540051168800500020001C630200000000000A
:10B2640000CEB30000406400CB42AB0001003200CA
:10B274000044A000CB22AB00010032000034A00047
:10B28400CB02AB00010032000024A000CAE2AB00F4
:10B29400010032000014A000CAC2AB000100320059
:10B2A4000004A0004F0478000000060000C0EB007A
:10B2B40080FF07000040EB00B6FF3700881F7800CE
:10B2C400804078000040EB00125E020000000000A5
:10B2D400004478000804E00001003200C222A80003
:10B2E400084078007052020000000000BE510200C5
:10B2F400000000000004E0000D0032006252020071
:10B3040000000000E14F400004003200084040000B
:10B3140070520200000000000500370010C0B300A6
:10B3240070520200000000004F0478000000060084
:10B334000804E000EDFF3A00D0D080000000E000F7
:10B344000A003A000080EB00D0D08800C202D50089
:10B354000080EA0061006000800040001016800058
:10B364000010A1000080700010168800D0D080006A
:10B374000000E900D0D08800DCFF3700889FBE00C1
:10B38400C222A800C9FF070045FF070047FF0700C6
:10B39400C1A12100804878000004E0009D00350030
:10B3A400F9FF3200E14F500004003A00BFFF0700EC
:10B3B4000E34020000000000F2FF3700E24F50009C
:10B3C40004003A00B9FF0700A24F02000000000089
:10B3D400ECFF3700E34F500004003A00B3FF0700CE
:10B3E4002C3C020000000000E6FF3700E44F500050
:10B3F4000E003200E54F500004003A00ABFF070096
:10B404000A47020000000000DEFF3700E64F50004C
:10B4140004003A00A5FF0700A0600200000000003D
:10B42400D8FF3700E74F500002003A009FFF0700A3
:10B43400D4FF3700EF4F500008003A0010C0B300AB
:10B444007052020000000000C222A9006A520200E9
:10B45400000000000000FE00CCFF3700F04F500059
:10B4640002003A000040EB0003003700F14F5000A7
:10B4740003003A0010C0B30090FF0700C3FF370079
:10B48400F24F500020003A001021EF001E21EF007F
:10B494009C21EF0000FE2F00CA06B6006001B30035
:10B4A4005036880001FF07000080FB000018A3004D
:10B4B4000100320010A1A8000008A300010032001E
:10B4C4001081A800F9FE07004804DD00F7FE07001C
:10B4D4000080FB0008047000D80C8800C80C8800A9
:10B4E40060002000E00C8800F0FE07004804DD0046
:10B4F400EEFE07000080FB00080070006008880072
:10B5040011E1A80006003700F34F500006003A008E
:10B514001021EF009C21EF0000FE2F00CA26B60088
:10B5240010C0B3003C003700F44F500008003A004C
:10B5340021E3A800C00020002262020000000000F5
:10B544000004780021E3A9004840DE00270037000A
:10B55400F54F500015003A0021E3A800C000200078
:10B564002262020000000000000478006A52020017
:10B57400000000004840DE0070520200000000009D
:10B58400084078007052020000000000BE51020022
:10B5940000000000E14F5000F0FF3A006252020048
:10B5A4000000000021E3A90078FF3700F64F5000A7
:10B5B40012003A00E43F0200000000000004BE0054
:10B5C4004808DE0070520200000000004048DE001F
:10B5D4000100200070520200000000004849DD0014
:10B5E4004840DE0000007100C848DE0070520200CE
:10B5F4000000000008407800070037000068A3003E
:10B6040002003200ABFE0700030037000040EB00ED
:10B6140001003700DFFE0700705202000000000046
:10B624005AFF3700829F2100004978000220200041
:10B63400E34F500004003A00D2CF880000082000F5
:10B64400E0CF880002003700D2CF8800E2CF880024
:10B65400E09F2100E1CF50000B00320003003900CD
:10B66400E2CF500017003A000E00370041C1B3008A
:10B674000148780041C6B300F09F210001487800DA
:10B6840021C3B3000C00370021C0B3000148780087
:10B69400A1C0B300F09F21000148780051C0B3005D
:10B6A4000500370012C0B3000248780052C0B3004E
:10B6B400F09F2100024878000000E800014878006B
:10B6C400000006000048EB00F09F21000048EB005A
:10B6D4000000E8000048EB0000000600829C210006
:10B6E400124178007041610004003A00CC22B70096
:10B6F4000080EA00C822B60001003700C822B70063
:10B704000180FB001C630400000000000080EA00CC
:10B71400CC22B600C822B6000180FB001C630400E2
:10B7240000000000889FBE008A1F78000045780052
:10B734000044EB0008003700F99F2100994078008D
:10B7440000102000E5FF0700994078000010200059
:10B75400EEFF07000844E8008A4F5400F6FF390062
:10B764004F0578004F04BE0000000600881F7800D3
:10B77400F89F21009840780000302000E3FF070084
:10B784009840780000102000D4FF0700984078000B
:10B7940000202000D1FF07000000EB004F047800D8
:10B7A40000000600889FBE00F09F210090407800B2
:10B7B40000302000C9FF070019002000CB02AB00B5
:10B7C40004003200591680000920B2008904E900FF
:10B7D400CF4CDE00F89F2100984078000020200024
:10B7E400CAFF07009840780000102000C7FF070038
:10B7F4009840780000202000B8FF07000900780076
:10B804004F04BE00000006000000E00003003A0000
:10B814000180EA00CC22B60007003700809C21009A
:10B82400104078007040600005003A000100780084
:10B83400CC22B7000180EA00C822B600020037001B
:10B8440001007800C822B7000280FB001C630400DA
:10B85400000000000080FB00E19F210011417800FE
:10B8640001042000E8FF37000080FB00E19F210075
:10B874001141780001102000E3FF37000080FB0035
:10B88400E19F210011417800D1CF8000DEFF370015
:10B89400881F78000080FB00E19F2100114178009F
:10B8A400D1CF8000D8FF0700F89F2100984078008E
:10B8B4000010200089FF0700984078000010200045
:10B8C40092FF07004F04780000000600889FBE0026
:10B8D4008A9FBE00719B21001185FB000A05E900C7
:10B8E400110020000A0DDD00000478008004EB0044
:10B8F4000E0037000A006400E19F21001141780026
:10B9040001202000C0FF0700FB9F21009B4078001E
:10B914000010200071FF07009B40780000102000F9
:10B924007AFF0700080444008904E800709B2100A2
:10B934001080FB00808F5400EEFF39004F05BE00DD
:10B944004F04BE0000000600C822B700000000003B
:10B954000000000000000000CA02B60000F0A700CA
:10B964000000EA000000EA004F00DE0000000600CC
:10B97400E0CF8000F4FF3700889FBE00C99F2100FC
:10B9840019007800F0FF07006384440098407800B1
:10B994000010200051FF070019007800EAFF07009B
:10B9A40080447800984078000010200057FF07007A
:10B9B400094078004F04BE0000000600889FBE00C6
:10B9C4008A9FBE0000202000DFFF07006044B8000B
:10B9D4000F003700FA9F21009A40780000102000E1
:10B9E4003EFF070000202000D7FF070080457800B5
:10B9F4009A4078000010200044FF07000804440027
:10BA04000B04E000010032000804E8008904E800A7
:10BA1400709B21001080FB00808F5400EDFF3900E3
:10BA2400080078004F05BE004F04BE000000060069
:10BA3400889FBE008A9FBE008C9FBE00719B210020
:10BA44009185FB008B05E900110020008B0DDD00C2
:10BA5400800478000004EB000005EB0015003700BB
:10BA64000B806400E19F2100114178000120200037
:10BA740065FF0700FC9F21009C4078000010200017
:10BA840016FF070000082000AFFF0700804678007B
:10BA94009C407800001020001CFF070089844400AB
:10BAA400080444000D04E000010032000804E8002A
:10BAB4000A05E800709B21001080FB00800F5500F0
:10BAC400E7FF3900080078004F06BE004F05BE00AE
:10BAD4004F04BE0000000600814F500004003A00ED
:10BAE4003100200080BB2000DE650400000000005F
:10BAF40051002000B0BB2000DE6502000000000001
:10BB040080A221001048E80000000600881F780089
:10BB14000044780041002000B0BA2000986502007B
:10BB240000000000501680004900DE006140600003
:10BB340088407800E8FF070031002000F0BA2000B8
:10BB44009865020000000000501680004800DE00E6
:10BB54006140600088407800DFFF0700410020005A
:10BB640020BB2000986502000000000050168000F1
:10BB74004700DE006140600088407800D6FF07007F
:10BB84002100200060BB2000986502000000000036
:10BB9400501680004600DE00614060008840780056
:10BBA400CDFF07004F04780000000600889FBE0008
:10BBB4008A1F78000004BE000205780080C2B3002A
:10BBC40070520200000000000800780022620200A7
:10BBD400000000000004780008007800CA52020047
:10BBE4000000000090C2B300705202000000000088
:10BBF4000000EB00890F5400040036001000200000
:10BC04008A0F5400010039000000EB0011C0B3009A
:10BC1400B1FF07004F0578004F04BE000000060086
:10BC2400889FBE008A1F7800804478000144780011
:10BC340080A221000048EB000904E00004003A005F
:10BC440050CF80000080A00050CF88000C00370047
:10BC54000804E0000A003200F103200050AE200086
:10BC6400DE6502000000000011012000A01921007F
:10BC7400DE650200000000006252020000000000C5
:10BC84004100200040B22000DE65020000000000F8
:10BC9400CB42A800C942A9003100200080B2200094
:10BCA4009865020000000000501680004A00DE0083
:10BCB4006140600011C0B30087FF0700CB42A900B8
:10BCC400C942A800C222A800C022A9008100200005
:10BCD400B0B220009865020000000000C202D50046
:10BCE4006140600011C0B3007BFF0700C222A900BD
:10BCF400C962A800CB62A9008100200030B32000F3
:10BD04009865020000000000501680004B00DE0021
:10BD14006140600011C0B3006FFF0700CB62A9004F
:10BD2400C962A90081002000B0B320009865020018
:10BD340000000000501680004B00DE0061406000EF
:10BD44008040EB0064FF0700C002A900C202A80003
:10BD54002000200048630200000000004100200091
:10BD640030B4200098650200000000001016800026
:10BD74006140600011C0B30057FF0700E1002000DC
:10BD840070B42000DE6502000000000021E3A8007A
:10BD94002100200050B5200098650200000000003A
:10BDA40072352000712B2000900020007FFF0700D7
:10BDB4000804E000080032003100200070B52000C3
:10BDC400986502000000000072352000712B2000ED
:10BDD400B000200075FF070041002000A0B520003E
:10BDE400986502000000000002252000011B2000CD
:10BDF400A00020006DFF07000804E00008003200E6
:10BE040031002000E0B52000986502000000000029
:10BE140002252000011B2000C000200063FF070052
:10BE240021E3A9008100200010B62000DE65020095
:10BE340000000000FAC32F00802C200010086500C9
:10BE440060168000003CB3006016880040062000A5
:10BE5400486302000000000010C0B3002BFF07007D
:10BE6400A100200090B62000DE6502000000000062
:10BE7400C02C2000100865000804E0000200320015
:10BE8400C962A800CB62A9004006200048630200F2
:10BE9400000000000040EB001CFF07000804E00065
:10BEA4000C003200A100200030B72000DE65020043
:10BEB4000000000040168000003CB30040168800DB
:10BEC40040062000486302000000000010C0B300D8
:10BED4000EFF07000904E000120032000804E0002D
:10BEE40010003200C002A900C202A800C422A800A7
:10BEF40001022000D0B72000DE650200000000002F
:10BF0400F1002000B0182100DE65020000000000EE
:10BF14006252020000000000C422A900C002A9006D
:10BF2400C202A900EA6102000000000061002000D2
:10BF3400D0B92000986502000000000088A221000A
:10BF440018407800825202000000000081002000A6
:10BF540030BA2000DE6502000000000050CF8000EF
:10BF64000080A10050CF8800184078004F05780069
:10BF74004F04BE0000000600CAC2A900CB22A900DB
:10BF8400CB02A900CB42A900CA02A900E24F50008B
:10BF940006003A00CAC2A800CB02A800CB22A8001F
:10BFA400CB42A800CA02A80005003700CAC2A900F3
:10BFB400CB02A900CB22A900CB42A900CA02A90046
:10BFC4000040E900E14F500006003E00C8C2A9004D
:10BFD400C922A900C902A900C942A900C802A9002E
:10BFE40005003700C8C2A800C922A800C902A800D9
:10BFF400C942A800C802A800C8E2A80000000600C0
:10C004000081FB008001EB0061015100E0815900D7
:10C01400EF0F5100E08F590035003E00026001002F
:10C024000F003700160037003100370024003700B6
:10C034002F0037002E0037002D0037002600370070
:10C044002B0037002A00370029003700280037006A
:10C05400270037002600370025003700100037007E
:10C06400C022A900E1806000818040001016800099
:10C074000010A10000807000101688000000060067
:10C084000104E00003003200C002A900C202A800BB
:10C0940000000600C002A900C202A90000000600B8
:10C0A4000104E00003003200C962A800CB62A900C9
:10C0B40000000600CB62A900C962A90000000600C6
:10C0C400E1806000501680000000A1000080700034
:10C0D4005016880000000600E1806000CA08DD00F8
:10C0E4005016800000A0A100008070005016880047
:10C0F4000000060080BB2800B053040000000000CC
:10C10400889FBE008A1F78000105780080047800AB
:10C114000004EB000400370039407800705202003C
:10C12400000000000804E8008A0F5400FAFF3900F8
:10C134004F0578004F04BE0000000600889FBE0033
:10C144008A1F7800F8CE80001000200050D18800AB
:10C15400E8FF070062520200000000000080FB00BC
:10C164008000EB00E80F5000E08F580087003E008D
:10C17400006001008C003700270037002A003700D8
:10C18400050037008100370059003700F0FF370001
:10C19400380037002D00370030C0B300004C780061
:10C1A40080C0B3001044980021E3A800C000200020
:10C1B4002262020000000000C800DE002144980052
:10C1C40030449800B0002000226202000000000009
:10C1D400C800DE004144980050449800A0002000AC
:10C1E4002262020000000000C800DE0061449800E2
:10C1F40070449800900020002262020000000000B9
:10C20400C800DE00014C9800104C980021E3A900FE
:10C21400A10020006100370062520200000000000B
:10C2240055FF0700CBFF37006252020000000000F8
:10C2340080447800625202000000000080407800D0
:10C24400094078006EFF0700C2FF37006252020007
:10C2540000000000804478006252020000000000E8
:10C26400C84CDD000080FB008904700059D18800AF
:10C27400B8FF3700625202000000000080447800DA
:10C2840030C0B300E1CF54000100320020C2B3003B
:10C294000C55020000000000625202000000000081
:10C2A400004578006252020000000000A1CAB300F9
:10C2B400814F550005003A0051C5B300814F50002D
:10C2C40002003A008984FB000400370020C2B30056
:10C2D4000C550200000000008004EB0070C0B300A5
:10C2E400004C780019449800210020002B003700EE
:10C2F4006252020000000000004578006252020011
:10C30400000000008560A900C854DD008080FB00A7
:10C314008984700001002200818F540001003600DE
:10C324008104780051C0B300014C78001A4498008D
:10C3340020449800310020000800780070FF0700B6
:10C34400F0CE800060CF8800E7804400C308DE00A0
:10C354008180400071CF88000001EB0082CF88000B
:10C36400418320008100400091CF8800A2CF880043
:10C37400B2CF88009560A80053D1800009017800ED
:10C38400B86702000000000072FF3700004CEB00A9
:10C394000040EB00104498001100200008007800D1
:10C3A40057FF07006BFF37004F0578004F04BE00AE
:10C3B40000000600809C210010417800F20050002B
:10C3C4008048EB0001CEB300014861000000060084
:10C3D400C922A800C902A800C8E2A800C8C2A800CF
:10C3E400C942A800C222A900C022A90000FE2F0051
:10C3F400CA26B600409E21000008EB00EDFF0700AE
:10C40400CB62A900C962A900C002A900C202A900A6
:10C414002D83A9002D43A9002D23A9002D63A90074
:10C4240000198000000EB300001988003023EF00CB
:10C4340020F02100201988002223EF0000000600CC
:10C44400401988002023A8002003A9002003AB0082
:10C45400FEFF3200001880000000060021E3A8005F
:10C46400C0002000F6FF0700CA52020000000000CE
:10C4740021E3A90000000600881F7800E1002000E5
:10C48400E0352000DE65020000000000F10020001D
:10C49400B0182100DE65020000000000F100200059
:10C4A400C036200098650200000000000000EB0088
:10C4B4000900370021E3A800C0002000E0FF0700C6
:10C4C4000004780021E3A900E0B92800B053020079
:10C4D4000000000008007800CA52020000000000BA
:10C4E40011002000B0372000986502000000000011
:10C4F400BE510200000000000004E000EDFF320025
:10C50400625202000000000040BA28009653020064
:10C51400000000004F04780000000600881F780027
:10C5240000047800709B210010407800EF4F500009
:10C5340005003E000080FB006F001000F1FF2700A3
:10C544000088DE000004640010CF8000E10F50007A
:10C554001200320005003900E20F50001B003200C7
:10C56400E30F500031003A0026003700809C210080
:10C5740001C2B30010C0600004003200080078005B
:10C58400B6540200000000002800370008007800BC
:10C59400E25402000000000024003700809C2100C7
:10C5A40001C2B30010C0600004003200080078002B
:10C5B400F2520200000000001C003700084078001E
:10C5C400825202000000000018003700809C210005
:10C5D40001C2B30010C060000600320008407800B9
:10C5E400705402000000000000C2B3007052020048
:10C5F40000000000084078007054020000000000B1
:10C604000A003700809C210001C2B30010C0600002
:10C61400030032004840DE007052020000000000B7
:10C624000840780070520200000000004F047800B7
:10C63400000006008000EB0011003700000000003D
:10C6440000000000000000000000000000000000E6
:10C6540000000000000000000000000000000000D6
:10C6640000000000000000000000000000000000C6
:10C674000000000000000000000000008100E8004D
:10C68400808F5000EDFF390000000600889FBE0037
:10C69400800478000004EB0009003700A00F20009C
:10C6A400E4FF0700A00F2000E2FF0700A00F200016
:10C6B400E0FF0700A00F2000DEFF07000804E800E9
:10C6C400890F5400F5FF39004F04BE000000060036
:10C6D4008001780002012000110020000000EB001E
:10C6E4000000400003826000010032000000A0004E
:10C6F400818040000201E900F9FF3A00719B2100AA
:10C7040091407800F0CF5000030032008180FB009C
:10C71400F08010000100DE0000000600C222A90023
:10C724006820EF006A20EF006020EF006220EF0035
:10C734001E21EF00F0FF2800AC20B6001C21EF0002
:10C7440000642000D00888000000210080D0880008
:10C754000000EB0090D0880000000600A1D080000B
:10C764000100E000040032000040EB00E28F5000C2
:10C7740030003E002B003700E24F50000F00320023
:10C7840005003E000004E0000A003200E14F5000C2
:10C7940021003A000C003700F14F50002400320011
:10C7A400F34F500022003200E44F50001A003A00C8
:10C7B40014003700D9FF07001000050041002000D5
:10C7C40060B7280011003700C222A8001E21EF0024
:10C7D4001621EF001421EF001E61A8008660A90055
:10C7E4009660A9006005800000C0A00000D0A100F0
:10C7F40000E0A100600588001000200090D08800AF
:10C804000400370051012000A0B728009A54020008
:10C81400000000000000050010002000A0D08800E7
:10C82400FCFF37000000EB00A0D0880000000600E9
:10C834000040EB0000000600881F780090D08000C4
:10C84400E10F500022003A008660AB0003003A007A
:10C854000040EB006200E2001E003A001FE1A80065
:10C864008780A90088D080000000EB000800370012
:10C87400521680004611DE00F1CE800082707800EE
:10C884008780AB00FEFF32008780A9000000E8002B
:10C89400880F5000F6FF39006220EF001E21EF00E0
:10C8A40006003700F0CE80000800400070F89700C2
:10C8B40070520200000000000804E9000800E000D3
:10C8C400F8FF3A0095FF070010C0B30001003700DD
:10C8D4000040EB004F047800000006004116800081
:10C8E400007C200001007000401688008BFF0700C8
:10C8F40020C0B30099FF0700BE51020000000000F1
:10C904000004E00005003200625202000000000052
:10C9140092FF07000004E00003003A00C6FF07008E
:0CC924000004E000F4FF320000000600F8
:020000040000FA
:10C93000901900002600000000000000161A0000F8
:10C940000400000000000000EC1900000C000000D2
:10C95000000000001A1A000004000000000000009F
:10C96000261A000002000000020000000300000080
:10C97000D01900000E00000000000000F8190000AF
:10C980000A000000000000000A1A00000600000073
:10C9900000000000DE1900000E0000000200000090
:10C9A000000800000000000000000000000000007F
:10C9B00000000000B61900001A000000000000008E
:10C9C0000008000000100000000000000018000037
:10C9D000D000000000000000281A00000200000043
:10C9E00000000000101A0000060000000000000017
:10C9F0001E1A00000400000000000000221A0000BF
:10CA00000400000000000000021A000008000000FE
:10CA1000000000002A1A00000200000000000000D0
:10CA2000D0180000C00000000200000092689200D0
:10CA3000689268009268820068726800926892004A
:10CA4000689268009268720068926800626862008A
:10CA50006852680038683800683868004A684400DE
:10CA6000684869005A00000000000000683968004A
:10CA7000397A39007A39DC003694360092689200AF
:10CA800068926800926872006892680062688A0022
:10CA900039423B006237020039643900F039E20064
:10CAA000365541005254000000000000664C6600FC
:10CAB0004CC04C00C04C00004CC04B00926892002F
:10CAC000689268009268720068926800626862000A
:10CAD00068B64E00284D7E004D9A4D00AA4D0000CC
:10CAE0004D4932004300000000000000902E70000D
:10CAF0002EB02E00B02E9A0031AC31009268920018
:10CB000068926800926872006892680062686200C9
:10CB100068563300402F5600318A3100DA30CC009D
:10CB20002E5350004900000000000000E86880001B
:020000040000FA
:10CB3000889FBE008A1F78000004780001057800F5
:10CB40008804780017003700320020001100090027
:10CB50008284D8000101780000004000E10F5100FC
:10CB60000600320061FE2100E20F51000800320091
:10CB7000008040001000BA000700370061FE21006D
:10CB8000008040001000BA004800DE0002003700BC
:10CB9000008040001080BA007052020000000000C7
:10CBA0008904E80008004500808F5400E6FF390042
:10CBB0004F0578004F04BE0000000600DCFF0700B0
:10CBC000E0BB280096530400000000001102200082
:10CBD00040272100F9FF0700C1042000502921004F
:10CBE000F6FF070061022000102E2100F3FF07006E
:10CBF0008102200070302100F0FF07005101200069
:10CC0000F0322100EDFF0700B10120004034210087
:10CC1000EAFF070081022000F0352100E7FF07004E
:10CC2000B101200070382100E4FF0700E10220007C
:10CC3000203A2100E1FF070051012000003D2100C2
:10CC4000DEFF070031022000503E2100DBFF07001D
:10CC5000E102200080402100D8FF0700C101200030
:10CC600060432100D5FF070011022000204521006C
:10CC7000D2FF0700C101200030472100CFFF07008D
:10CC800051022000F0482100CCFF070011022000D3
:10CC9000404B2100C9FF070091012000504D2100A9
:10CCA000C6FF0700F1012000E04E2100C3FF07008E
:10CCB00091022000D0502100C0FF07005102200047
:10CCC00060532100BDFF070061032000B055210023
:10CCD000BAFF0700E103200010592100B7FF370019
:10CCE000881F7800E10020007091200090FF07006D
:10CCF0006252020000000000004478000840780002
:10CD00007052020000000000E0BB280096530200B1
:10CD100000000000F80DB2009885B2000804E90098
:10CD20004F40DE004F047800000006000400FA00C7
:10CD3000881F7800F0FF2F0001002000D0BF9F0067
:10CD4000E1BF9F004507A9002CA3EF004227A900DF
:10CD50005FB89700EFB8970061015000E08158007C
:10CD6000D2BF9F00E3BF9F00E00F5000E08F58004C
:10CD7000F7FF3A0000FE2F0023358000830060009B
:10CD80005100B30021358800C406B6003000B3005E
:10CD90002036880088C0B300009E21000848780033
:10CDA0000080E8000008EB00EA61020000000000DB
:10CDB000965102000000000068C0A80068E0A800CA
:10CDC0008000EB00F00F2000825102000000000004
:10CDD00030CF880021002000F00F20008251020097
:10CDE0000000000040CF880051168000C208DE001D
:10CDF000E380600032BB2800A09E210062C878005A
:10CE000068C0A90068E0A90050CF80000080A100A0
:10CE100050CF8800709B2100084878003260EF00F6
:10CE200020BB28009653020000000000E60F02001D
:10CE3000000000004F0478000080FA0000000600A7
:10CE4000BAFF070090130200000000000000050078
:10CE5000E1806000C908DD00F5DF2F007616800054
:10CE600086826200858270007516880001FE2F00A0
:10CE700035358000858060007100B3003135880051
:10CE8000F50F2E0046368000868262000150200099
:10CE90008580700041368800C01188003022EF0084
:10CEA0003062A800610161004410DD00F1FE2F0036
:10CEB00085118000858060008100700081118800EC
:10CEC000E38161008381410090FF2F003002B600B2
:10CED000008071008011880061026200E0FF2F0075
:10CEE0003002B60000007200801188003222EF008C
:10CEF0004E11DD00F0FF2B003202B6000000710081
:10CF0000901188000000060031E2A8003342A8001A
:10CF100087C0A900C922A9000000060031E2A900CB
:10CF20003342A90030358000F001B300303588006D
:10CF3000F00F2E00C826B600CF22A900C922A800F3
:10CF4000000006003322AB00FEFF3A00A01188006B
:10CF5000000006003202AB00FEFF3200B01180007C
:10CF60000000060090118000614060000000060093
:10CF7000889FBE008A9FBE008C1F78008002EB0055
:10CF80000203E900800378000104780003067800BA
:10CF9000A92C20009A0020006B00200070CF800098
:10CFA000E48242000028E60005007800F019E30062
:10CFB000FEFF350037017800B70178000280FD00E0
:10CFC00003026900F40FB200040169008481690062
:10CFD0000280FD00F00020000030E600060078002E
:10CFE000800078000C800900000000001980A1007A
:10CFF0000281D3001950AD008381D3001958AD00D0
:10D000000C800900000000001980A0001970A30026
:10D010000482D3008100E900F2FF3100EF0010002C
:10D020000122DE00041C78004300DE000000E8005E
:10D03000F639B4009580AB0006003200A0CF800026
:10D04000F619E30003003200F219B4001000780072
:10D050002011880070035300D0FF31004F06780084
:10D060004F05BE004F04BE001C5504000000000028
:10D0700081C0B300709B210001487800710040001E
:10D080001054A1000000060000BC280096530400C4
:10D09000000000000101200040062100DE650400C0
:10D0A0000000000011022000203F2000DE65020089
:10D0B0000000000011C0B300408821000148780042
:10D0C0000000060011022000203F2000DE65020063
:10D0D0000000000011C0B300408821000148780022
:10D0E0000000050011022000203F2000DE65020044
:10D0F0000000000011C0B300408821000148780002
:10D100000000050011022000203F2000DE65020023
:10D110000000000011C0B3004088210001487800E1
:10D120000010050011022000203F2000DE650200F3
:10D130000000000011C0B3004088210001487800C1
:10D14000000006000080FB000038A300030032004E
:10D15000C002A900C202A80002003700C002A90054
:10D16000C202A9000028A30003003200C962A8007F
:10D17000CB62A90002003700CB62A900C962A900F6
:10D180000018A30003003200C942A900CB42A80046
:10D1900002003700C942A900CB42A9000008A30041
:10D1A00008003200809C2100104078007040600030
:10D1B00002003200C8C2A80000000600CCC2A800CD
:10D1C00001003700CCC2A900C8C2A90000000600B7
:020000040000FA
:04D1D000000000005B
:020000040000FA
:020000040001F9
:0457F800DFF90000D5
:020000040000FA
:020000040001F9
:0457FC007F3F0000EB
:00000001FF
